:020000040007F3
:1010000000B20020D5130700DD130700DF1307002F
:10101000E1130700E3130700E513070000000000D9
:10102000000000000000000000000000C1130700E5
:10103000E913070000000000EB130700ED130700A1
:10104000EF130700EF130700EF130700EF1307007C
:10105000EF130700EF130700EF130700EF1307006C
:10106000EF130700EF130700EF130700EF1307005C
:10107000EF130700EF130700EF130700EF1307004C
:10108000F92B0700EF130700EF130700EF1307001A
:10109000EF130700EF1307005D280700EF130700A9
:1010A000EF130700EF130700EF130700EF1307001C
:1010B000EF130700EF13070000000000000000001E
:1010C000EF130700EF130700EF130700EF130700FC
:1010D00059270700EF130700EF1307000000000077
:1010E0000000000000000000000000000000000000
:1010F00000000000000000000000000000000000F0
:1011000000000000000000000000000000000000DF
:1011100000000000000000000000000000000000CF
:1011200000000000000000000000000000000000BF
:1011300000000000000000000000000000000000AF
:10114000000000000000000000000000000000009F
:10115000000000000000000000000000000000008F
:10116000000000000000000000000000000000007F
:10117000000000000000000000000000000000006F
:10118000000000000000000000000000000000005F
:10119000000000000000000000000000000000004F
:1011A000000000000000000000000000000000003F
:1011B000000000000000000000000000000000002F
:1011C000000000000000000000000000000000001F
:1011D000000000000000000000000000000000000F
:1011E00000000000000000000000000000000000FF
:1011F00000000000000000000000000000000000EF
:10120000DFF80CD000F04EF900480047254E0700EB
:1012100000B2002030B450E8012F93B2C4892344B7
:101220008489A34228BF1B1B0489A34202BFBFF3CA
:101230002F8F002007E0C3EA020340E80134002CAE
:10124000E9D14FF001000A6030BC704750E8012F2F
:10125000C2EA024240E801210029F7D1704730B4C8
:1012600050E8022F1FFAA2F3C488A34202BFBFF3C3
:101270002F8F00200DE0C48923448489A34228BF16
:101280001B1BC2EA034340E80234002CE8D14FF0B4
:1012900001000A6030BC704750E8022FC2EA2242C7
:1012A00040E802210029F7D17047034653E8022F96
:1012B000D988B2EB324F4FF0000017BF92B241EA2B
:1012C000014142EA014104E05A68B2EB324F08BFE3
:1012D000012043E80212002AE8D1704730B40446E6
:1012E00054E8000F0D4644E80053002BF8D1156078
:1012F00030BC704730B4044654E8000F40EA0105A2
:1013000044E80053002BF7D1156030BC704730B46F
:10131000044654E8000F00EA010544E80053002B9E
:10132000F7D1156030BC704730B4044654E8000F64
:1013300080EA010544E80053002BF7D1156030BC6A
:10134000704730B4044654E8000F00EB010544E850
:101350000053002BF7D1156030BC704730B4044601
:1013600054E8000FA0EB010544E80053002BF7D12F
:10137000156030BC704770B404464FF0000054E86C
:10138000006F0D68AE4207BF44E80023012044E827
:1013900000630E60002B1CBF0020F0E770BC70479C
:1013A00030B4044654E8000F88422CBF451A054665
:1013B00044E80053002BF5D1156030BC70470000A5
:1013C0001EF0040F0CBFEFF30880EFF3098007F065
:1013D00005BC00000648804706480047FEE7FEE7D8
:1013E000FEE7FEE7FEE7FEE7FEE7FEE7FEE7FEE7D5
:1013F0006128070001120700202A04DB203A00FAC6
:1014000002F1002070479140C2F1200320FA03F35B
:1014100019439040704700000048704700BE070025
:1014200040EA01039B0703D009E008C9121F08C066
:10143000042AFAD203E011F8013B00F8013B521EE6
:10144000F9D27047D2B201E000F8012B491EFBD25D
:1014500070470022F6E710B513460A4604461946BF
:10146000FFF7F0FF204610BD421C10F8011B0029B9
:10147000FBD1801A704730B504460020034600E0D7
:101480005B1C934203D2E05CCD5C401BF8D030BDC6
:10149000034611F8012B00F8012B002AF9D1184658
:1014A00070470000064C074D06E0E06840F001037D
:1014B00094E8070098471034AC42F6D3FFF7A4FE37
:1014C00000CE070020CE07002DE9F0438BB0804608
:1014D000129D15F9046B009614461F4689462B464B
:1014E00002A81146424600F0BCFC02A80146129A2E
:1014F00000F0A7FC4046414602AA129B00F091FC76
:101500002046214602AA129B00F08BFC2B4638464F
:1015100039464A46009600F0A4FC02A83946129AC1
:1015200000F08FFC02A8014642462B46009600F0D0
:1015300098FC02A8014622462B46009600F091FC3A
:101540002046214642462B46009600F08AFC48463B
:1015500049462246129B00F064FC2046414602AAFE
:101560002B46009600F07DFC384639462246129BF9
:1015700000F057FC384639464A462B46009600F0A4
:1015800070FC204602A9324600F035FE0BB0BDE8E3
:10159000F083F0B589B01C4607460E4615466846EE
:1015A00011461A4600F04DFC384639466A46234635
:1015B00000F037FC684669462A46234600F031FCB5
:1015C000304631466A46234600F02BFC09B0F0BD98
:1015D0001AB1013A8B5C8354FAE770472DE9F04762
:1015E0008846B3F902101F460825CB1D202493FB23
:1015F000F5F51F31954291FBF4F44FFA84F928BFB9
:1016000015460646494600F077FA2A4630464146D6
:10161000FFF7DEFFB7F90230ED009D4220D9ED1A49
:1016200006EB840100228E420AD251F8040D20FA02
:1016300005F313430B60C5F1200300FA03F2F2E750
:101640002437384631464A4600F062FA012807D06E
:10165000304631463A464B46BDE8F04700F020BFE1
:10166000BDE8F0872DE9F04793F9006092B0044699
:101670008946104631461546984600F073FA002810
:1016800040F0978002A84946424600F0DAFB434604
:101690000AA8214602AA00F0C4FB02A8014642465D
:1016A00000F0CFFB4346484649462A4600F0B9FBC6
:1016B00008F1040728462946424600F0C2FB2046AE
:1016C00021462A463B46009600F0FAFA284629466B
:1016D0002A463B46009600F0F3FA284621462A4661
:1016E0003B46009600F0BDFB204621462A46434675
:1016F00000F097FB2846214622463B46009600F024
:10170000DFFA20463B46009621462A4600F0D8FAEA
:101710002368DB07204613D5334621463A4600F0BE
:10172000BFF931468246204600F058FD06F180435D
:10173000013B54F8230040EACA7044F8230002E059
:10174000314600F04BFD28462146424600F079FB29
:10175000284629460AAA3B46009600F082FB284606
:1017600029460AAA3B46009600F07BFB0AA80146E0
:101770002A463B46009600F074FB204621460AAA02
:10178000434600F04EFB02A802463B462146009627
:1017900000F067FB20462946324600F02CFD284623
:1017A0004946324600F027FD484602A9324600F07D
:1017B00022FD12B0BDE8F0870048704750CD070009
:1017C0002DE9F04FEFB01E46789C059023780493E6
:1017D000B4F9023092461F33202293FBF2F3DBB2BE
:1017E00006939DF9187094F9012007F1FF3926AB93
:1017F000002543F829506EAB03EB89034EA88B46B6
:10180000314643F8805C43F8605CFFF7E1FE94F9F1
:10181000012056A8B118FFF7DBFE9DF910604EA815
:10182000314600F09FF98046002840F02F8156A8ED
:10183000314600F097F90546002840F0258104F173
:10184000240840464EA93A4600F062F9012840F0CB
:101850001D81404656A93A4600F05AF901280890E1
:1018600040F014813B461EA856A9424600F041FABA
:101870000DF1380C60465946524623464CF8295023
:10188000CDF80CC0FFF7AAFEDDF80CC0009760464B
:1018900061461EAA4346CDF824C00DF5BC7900F080
:1018A000AEFA4346009716A84EA91EAA00F0A7FA62
:1018B00048463246059900F09EFCB300039309EBBD
:1018C000030B039A059B58469918324600F093FC87
:1018D00004F144031946324636A8079300F08BFC06
:1018E00004EB860132463EA8443104F1040A00F0BC
:1018F00082FC494600961EA836AA534600F0B1FA6B
:101900004A465B4636A83EA90094FFF7DDFD1EA8B7
:1019100001463346524600F0ECF91EAA48465946A5
:101920002346FFF736FEDDF824C0079B0B93604685
:10193000059B0C933946CDF814C00A95CDF8349028
:1019400000F02AFC3946054616A800F025FCA842FE
:10195000B8BF284685B2DDF814C06F1E3FB260469E
:10196000394600F0CDFD394610F1000916A818BF20
:101970004FF0010900F0C4FD002814BF022300232A
:1019800043EA09090DF1280B32465BF8297026A8B5
:10199000394600F030FC039B3246F9182EA800F0BF
:1019A0002AFC31461EA800F0A7F8023D089B1E93B2
:1019B000AEB237B2002F44DB23461EAAD4F8A4509F
:1019C00026A82EA9A84739460EA800F099FD394649
:1019D000051C16A818BF012500F092FD002814BFB1
:1019E000022300231D430AAB53F8257037B39DF93A
:1019F000105036A839462A4600F0FDFB039B3EA84E
:101A0000F9182A4600F0F7FB36A83EA91EAA23467D
:101A1000FFF7BFFD46A826A936AA5346009500F059
:101A200020FA36A83EA926AA2EAB0094FFF74CFD5B
:101A30001EA8014646AA234600F0F3F9013EB6B2BD
:101A4000B7E79DF910501EA8014652462B4600F0FC
:101A500050F9234626A82EA91EAAFFF79AFD9DF944
:101A60001840404626A9224600F052F8012805D029
:101A700026A801464246234600F012FD26A84EA99C
:101A80002A4600F05AF802E0404600E028466FB0CF
:101A9000BDE8F08F00000000000000000000000022
:101AA000C3F10803DB0070B501330446002003A531
:101AB0005B1920C940CAAD1920C4184720C940CAC3
:101AC000754120C420C940CA754120C420C940CAFC
:101AD000754120C420C940CA754120C420C940CAEC
:101AE000754120C420C940CA754120C420C940CADC
:101AF000754120C4404170BD10B5002253B28B42E5
:101B000005DA1BB2002440F823400132F6E710BD8D
:101B100010B5013AD2B253B2002B09DB1BB250F818
:101B2000234051F823309C4204D8F2D2FF2002E037
:101B3000002000E0012040B210BD013A30B5D2B221
:101B4000002453B2002B09DB1BB2013A51F8235099
:101B500050F823306B401C43D2B2F2E7B4FA84F061
:101B6000400930BD10B500231A465CB28C4204DA3D
:101B700050F8244001332243F7E7B2FA82F04009DB
:101B800010BD00002DE9F043A3B09846019112ABBF
:101B90004146074610469146009300F0FDFAC0EB1F
:101BA000881086B2454C33B21C40002CBEBF04F1F5
:101BB000FF3464F01F040134202593FBF5F5EDB2EA
:101BC0006DB2A4B202A8294624B2FFF795FF28B24D
:101BD00002AB002C03EB800010DD002213464345CE
:101BE00010D259F8235005FA04F10A4340F8232093
:101BF000C4F1200225FA02F20133F0E749464246D9
:101C000000F0F9FA0FFA88F502AB4FEA4509012412
:101C100003EB8505330444D40022114653B24B45EF
:101C200022DA0DF1880E0EEB840E0DF1880C18B23D
:101C30005EF888EC0CEB83035EF820E053F8803C00
:101C4000C3EB0E035B1A734502D08CBF0121002148
:101C5000C4F1010E0DF1880C0CEB8E0E01325EF812
:101C600088EC4EF82030D9E7621A544202A8414667
:101C7000544100F0B3FA22AA08F1FF3302EB8303C8
:101C800002EB8802284652F8801C53F8802C013E53
:101C900042EAC172414643F8802CB6B200F09EFA87
:101CA000B8E722AB03EB8404384654F8881C42465C
:101CB00000F0A1FA23B0BDE8F08300BF1F00008050
:101CC00070B59DF910401D4623460646FFF7E8FE15
:101CD00030B9284631462246FFF71AFF012807D0BF
:101CE000304631462A462346BDE8704000F0D8BB56
:101CF00070BDF0B50646A1B00F4608461946154618
:101D00001C46FFF72FFF20B130462146FFF7F4FEB7
:101D100073E068463946224600F06DFA08A8294665
:101D2000224600F068FA10A82146FFF7E5FE0123DD
:101D300018A821461093FFF7DFFE684608A922463F
:101D4000FFF7E6FE002853D0009BDA0704D468466C
:101D5000214600F043FA26E0089BDB0704D408A8DC
:101D6000214600F03BFA3DE000281EDD08AA23468C
:101D70006946684600F094FB6846214600F02EFA5A
:101D800010A818A92246FFF7C3FE002805DA10A8FC
:101D900001462A462346FFF783FE10A8014618AAEB
:101DA000234600F07DFB10A81DE008A86A462346E4
:101DB000014600F075FB08A8214600F00FFA18A8AC
:101DC00010A92246FFF7A4FE002805DA18A801464C
:101DD0002A462346FFF764FE18A8014610AA2346A8
:101DE00000F05EFB18A82946224600F06BFCA4E731
:101DF000304610A9224600F0FEF921B0F0BD70B5C2
:101E000090B006469DF950401D466846234600F0B6
:101E10003AF8304669462A462346FFF7B3FE10B02B
:101E200070BD30B51C4691B0054693F90030684648
:101E300000F029F8D4F8AC3028466946984711B02C
:101E400030BD30B5144691B0054692F90020684681
:101E500000F0DEF9D4F8AC3028466946984711B056
:101E600030BD70B59DF910401D462346064600F072
:101E700017FB38B1304631462A462346BDE870404C
:101E8000FFF70EBE70BD2DE9F04F08B4F8CA04B4D8
:101E900051F8042BA3FB028940F8048B4FF0000A91
:101EA000E4FB629A4FF0000BE5FB62AB4FF0000CD5
:101EB000E6FB62BC4FF0000EE7FB62CE51F8042B4C
:101EC0004FF00008E3FB628940F8048BE4FB629A60
:101ED000E5FB62ABE6FB62BCE7FB62CE51F8042B8C
:101EE0004FF00008E3FB628940F8048BE4FB629A40
:101EF000E5FB62ABE6FB62BCE7FB62CE51F8042B6C
:101F00004FF00008E3FB628940F8048BE4FB629A1F
:101F1000E5FB62ABE6FB62BCE7FB62CE51F8042B4B
:101F20004FF00008E3FB628940F8048BE4FB629AFF
:101F3000E5FB62ABE6FB62BCE7FB62CE40F8049BCC
:101F400040F804AB40F804BB40F804CB40F804EB85
:101F50000CBC052B00F01E810C68A0F11400A1F14F
:101F60001401A2F1140252F804EB4FF0000550F8EE
:101F7000046BE4FB6E5652F804EB50F8047BE4FB70
:101F80006E6752F804EB50F8048BE4FB6E7852F85D
:101F900004EB50F8049BE4FB6E8952F804EB50F814
:101FA00004ABE4FB6E9AA0F1140052F8044B51F814
:101FB00004EB4FF0000CE4FB6EC540F804CB51F885
:101FC00004EBE4FB6E5640F8045B51F804EBE4FBD1
:101FD0006E6740F8046B51F804EBE4FB6E7840F850
:101FE000047B51F804EBE4FB6E8940F8048B51F854
:101FF00004EBE4FB6E9AA0E80006062B00F0CA8012
:102000000C68A0F11800A1F11801A2F1180252F811
:1020100004EB4FF0000550F8046BE4FB6E5652F8E9
:1020200004EB50F8047BE4FB6E6752F804EB50F8C5
:10203000048BE4FB6E7852F804EB50F8049BE4FB4D
:102040006E8952F804EB50F804ABE4FB6E9A52F838
:1020500004EB50F804BBE4FB6EABA0F1180052F89F
:10206000044B51F804EB4FF0000CE4FB6EC540F854
:1020700004CB51F804EBE4FB6E5640F8045B51F8D6
:1020800004EBE4FB6E6740F8046B51F804EBE4FBEF
:102090006E7840F8047B51F804EBE4FB6E8940F85D
:1020A000048B51F804EBE4FB6E9A40F8049B51F862
:1020B00004EBE4FB6EABA0E8000C072B6AD008B47D
:1020C0000C68A0F11C00A1F11C01A2F11C0252F845
:1020D00004EB4FF0000550F8046BE4FB6E5652F829
:1020E00004EB50F8047BE4FB6E6752F804EB50F805
:1020F000048BE4FB6E7852F804EB50F8049BE4FB8D
:102100006E8952F804EB50F804ABE4FB6E9A52F877
:1021100004EB50F804BBE4FB6EAB52F804EB50F850
:1021200004CBE4FB6EBCA0F11C0052F8044B51F848
:1021300004EB4FF00003E4FB6E3540F8043B51F82C
:1021400004EBE4FB6E5640F8045B51F804EBE4FB4F
:102150006E6740F8046B51F804EBE4FB6E7840F8CE
:10216000047B51F804EBE4FB6E8940F8048B51F8D2
:1021700004EBE4FB6E9A40F8049B51F804EBE4FB9B
:102180006EAB40F804AB51F804EBE4FB6EBCA0E886
:10219000001808BCBDE8F08F0139C9B24BB2002B62
:1021A0000BDA013111F0FF0315D059B201F1804370
:1021B000013B50F82320002304E050F82330002B8B
:1021C000EAD0EEE712B152080133FBE7481E03EBF9
:1021D000401080B200E0184600B2704700EB810169
:1021E0000023884206D251F8042D43EA52030B60C3
:1021F000D307F6E7704730B5002463B2934206DA9E
:102200001BB2013451F8235040F82350F5E730BD9C
:102210002DE9F04FB1E8005E06B4AAFB09124FF0B9
:102220000003EBFB69234FF00004ECFB69344FF033
:102230000005EEFB69454FF00006EBFB6A63ECFB23
:102240006A344918524176415B41A9FB09784FF045
:10225000000949F1000918EB0108A0E88001AAFB78
:102260000A78574158EB0608A0E88001EEFB6A4562
:102270004FF0000A4AF1000A4FF00001ECFB6B142A
:10228000EEFB6B454FF00002EEFB6C255FEA59094F
:102290004941644152416D4149F10009EBFB6B3A00
:1022A0001AEB010AA0E80804ACFB0C6A66415AEB81
:1022B000020AA0E84004AEFB0E6A6E415AEB090A1E
:1022C000A0E8400406BC052A00F0E680A0F1140056
:1022D000A1F11401B1E8E043A5FB0E344FF0000575
:1022E000E6FB6E454FF00006E7FB6E564FF0000729
:1022F000E8FB6E674FF00008E9FB6E784FF00009CD
:10230000DB1864416D4176417F4158EB080859F173
:10231000000950F804CB13EB0C0350F804CB54EB3A
:102320000C0450F804CB55EB0C0550F804CB56EBDD
:102330000C0650F804CB57EB0C0758F1000859F184
:102340000009A0F11400EEFB0E89A0E8F803062AAC
:1023500000F0A280A0F11800A1F11801B1E8E04757
:10236000A5FB0E344FF00005E6FB6E454FF000066E
:10237000E7FB6E564FF00007E8FB6E674FF0000872
:10238000E9FB6E784FF00009EAFB6E894FF0000A16
:10239000DB1864416D4176417F4158EB080859EBE9
:1023A00009095AF1000A50F804CB13EB0C0350F85A
:1023B00004CB54EB0C0450F804CB55EB0C0550F84F
:1023C00004CB56EB0C0650F804CB57EB0C0750F837
:1023D00004CB58EB0C0859F100095AF1000AA0F19E
:1023E0001800EEFB0E9AA0E8F807072A54D0A0F1D7
:1023F0001C00A1F11C01B1E8E04FA5FB0E344FF029
:102400000005E6FB6E454FF00006E7FB6E564FF009
:102410000007E8FB6E674FF00008E9FB6E784FF0AD
:102420000009EAFB6E894FF0000AEBFB6E9A4FF051
:10243000000BDB1864416D4176417F4158EB080881
:1024400059EB09095AEB0A0A5BF1000B50F804CB6F
:1024500013EB0C0350F804CB54EB0C0450F804CBF2
:1024600055EB0C0550F804CB56EB0C0650F804CB9A
:1024700057EB0C0750F804CB58EB0C0850F804CB82
:1024800059EB0C095AF1000A5BF1000BA0F11C009A
:10249000EEFB0EABA0E8F80FBDE8F08F00000000E7
:1024A000C3F10803DB0070B50133002403A500BFAE
:1024B0005B1920C940CAAD1B20C0184720C940CABB
:1024C000B54120C020C940CAB54120C020C940CA7A
:1024D000B54120C020C940CAB54120C020C940CA6A
:1024E000B54120C020C940CAB54120C020C940CA5A
:1024F000B54120C06441B4FA84F0400970BD00BF0A
:102500004A11012301F01F0150F822008B401840AE
:1025100070470000F0B50C4689B008220646FFF768
:102520006AFEE36A0393236B0493636B0593A36BC7
:102530000693E36B0793002769466A4608236846BB
:10254000029701970097FFF7ABFA314605466A46B6
:1025500008233046FFF7A4FA236B0393636B0493BD
:10256000A36B0593E36B0693054469466A4608230B
:1025700068460797FFF794FA314605446A460823F0
:102580003046FFF78DFA236A0093636A0193A36ACA
:102590000293A36B0693E36B0793054431466A46A7
:1025A00008233046059704970397FFF779FA636A83
:1025B0000093A36A0193E36AA26B0293636B039394
:1025C00004920693E26B236A059205440793314611
:1025D0006A4608233046FFF763FAE36A0093236BE9
:1025E0000193636B0293236A0693A36A07930544DE
:1025F00031466A4608233046059704970397FFF74C
:102600004FFF236B0093636B0193A36B0293E36B08
:102610000393636A0693E36A07932D1A31466A4669
:102620000823304605970497FFF73AFF636B009342
:10263000A36B0193E36B0293236A0393636A04938E
:10264000A36A0593236B07932D1A31466A46082324
:1026500030460697FFF724FFA36B0093E36B0193CB
:10266000636A0393A36A0493E36A0593636B079316
:102670002D1A314630466A46082302970697FFF71F
:102680000FFF2D1A16D5304631460D4A0823FFF7A5
:1026900007FA4519F7D410E0094831460822FFF738
:1026A00037FA012809D030463146054A0823FFF79A
:1026B000F7FE2D1A002DEFD0F5E709B0F0BD00BFF1
:1026C00054CD0700F8B5036813F0010506460F4620
:1026D000144605D001463A462346FFF7E1F9054680
:1026E00030462146FFF77AFD45B104F18042013AB8
:1026F00056F8223043F0004346F82230F8BD2DE969
:10270000F04115468AB00446884602A800212022DE
:10271000FEF7A1FE2E780323204641462A462F1DB0
:1027200076B20293FFF78DFB2046214602AA3B4674
:102730000096FFF796FB2046214642462B46FFF7C0
:1027400070FB00962046214605F184023B46FFF7C8
:10275000B7FA0AB0BDE8F0812DE9F0411E4E4FF402
:102760008271D6F8040130B11C48C268521CC260A4
:10277000304605F057FF00254FF4A07707EB8501A1
:102780008AB23046B25812B389B205F04BFF1348F3
:10279000103000EB0514204608F074FD1048114974
:1027A0002246401AC008042101EB00400EA105F0AA
:1027B000F5FC616819B1204608F0BAFC07E0A16891
:1027C00011B1204608F0B4FC206800B180476D1CB0
:1027D000022DD3D3BDE8F0810040024070590020A3
:1027E00088CE070038CE070074696D65725F666930
:1027F00072652028307825782900000000F00CBA96
:1028000070B50E46144900EB400001EBC0051446BC
:10281000E86A183520B101280FD0022805D113E04D
:10282000284600F02FFAA04201D2002411E02246EF
:102830003146284600F060FA0BE0284600F022FA04
:10284000A042F4D20446F2E73146284600F025FAC9
:102850000446204670BD00007491002006F0BCB80C
:10286000F0B5D34AD3494FF080541368D4F83001FF
:102870000978D4F83421451CC1F3031107D08446EC
:10288000164601270025BCF1060F04D013E003F023
:10289000FF0C0E46F5E7032E05D0042E03D0052EBF
:1028A00001D0062E07D1B4F82463DFF80CC3C6F3B9
:1028B0000426CCF80060DEB2062E06D1032904D12E
:1028C000DFF8FCC2BD4ECCF87460461C06D08446CE
:1028D0004FEA0206BCF1060F04D013E003F0FF0C30
:1028E0000E46F7E7032E05D0042E03D0052E01D0A7
:1028F000062E07D1D4F84462DFF8C8C2C6F34236C8
:10290000CCF80060DEB2062E08D1032906D1AE4E07
:10291000D6F800C02CF0807CC6F800C0461C05D05C
:1029200084461646BCF1060F04D014E003F0FF0CF9
:102930000E46F7E7032E05D0042E03D0052E01D056
:10294000062E08D14FF08046C6F80C51C6F810513B
:102950009C4E361F3560DEB2062E08D1032906D103
:10296000DFF860C203260CF1640CCCF80060DEB224
:10297000062E11D103290FD1DFF850C20526CCF85D
:102980000060924E78363760904E083635600CF114
:10299000040C3F26CCF80060461C05D08446164641
:1029A000BCF1060F04D087E003F0FF0C0E46F7E7FA
:1029B000032E7CD0042E7FD0052E01D0062E7BD195
:1029C000834E3668DFF80CC2CCF80060804E361DAE
:1029D00036680CF1040CCCF800607D4E0836366881
:1029E0000CF1040CCCF80060794E0C3636680CF112
:1029F000040CCCF80060764E103636680CF1040CEE
:102A0000CCF80060724E143636680CF1040CCCF829
:102A100000606F4E18363668DFF8B8C10CF1200C34
:102A2000CCF800606A4E1C3636680CF1040CCCF809
:102A30000060674E203636680CF1040CCCF800605C
:102A4000634E243636680CF1040CCCF80060604EFE
:102A5000283636680CF1040CCCF800605C4E2C363D
:102A600036680CF1040CCCF80060594E30363668EC
:102A7000DFF860C10CF1400CCCF80060544E3436E5
:102A800036680CF1040CCCF80060514E38363668CC
:102A90000CF1040CCCF800604D4E3C3636680CF15D
:102AA000040CCCF800604A4E4036366800E003E083
:102AB0000CF1040CCCF80060461C05D08446164688
:102AC000BCF1060F04D011E003F0FF0C0E46F7E74F
:102AD000032E05D0042E03D0052E01D0062E05D1DD
:102AE000D4F858423C4E04F04F043460441C04D0E7
:102AF00003461146062B02D010E0DBB2FAE70329A9
:102B000005D0042903D0052901D0062906D133496F
:102B10000B68DB0702D06FF001030B6006280CD1B5
:102B2000032A0AD0042A08D0052A06D0062A04D18E
:102B30002B48016841F480610160234874380168C2
:102B400041F470010160BFF34F8FBFF36F8F4FF0FF
:102B50001021D1F80002002803DBD1F8040200287C
:102B600022DA204A176020480368002BFCD0152386
:102B7000C1F800320468002CFCD0C1F804320168AE
:102B80000029FCD0156001680029FCD0BFF34F8FED
:102B90000D48F0380168154A01F4E0611143016005
:102BA000BFF34F8F00BFFDE7124911480860F0BD29
:102BB000E00F00F0E80F00F0403501400DF0ADBA35
:102BC00000C007403C050040FCED00E0105600400E
:102BD0000404001020C50040E40E00400004004042
:102BE0003C17004004E5014000E401400400FA0500
:102BF0000090D0036C5A0020064808B500210160FF
:102C00000068009005F07EFB05F054F90028FBD128
:102C100008BD00000001014010B5124C02202061E7
:102C2000606111A0A06104F17800E0614FF4805070
:102C300020620020A06260620BA1A164E0620D49E5
:102C4000E1641021A065C4E91410E0650AA1E01D4B
:102C5000FEF71EFC09A12046FEF71AFC2020A071F9
:102C600010BD0000749100205465726D696E616C36
:102C700000000000ECA10020525454005345474787
:102C8000455200000269C1688A4203D88068401A30
:102C9000104400E0501A401E70472DE9F047C46808
:102CA0001746894606464FF000083069A04201D910
:102CB000051B02E0B168201A0D1A6D1E00D1012516
:102CC000B068001BA84200D80546BD4200D33D466F
:102CD00070682A4620444946FEF7A2FBB0687F1B75
:102CE0002C44A844A944A04200D10024F460002F41
:102CF000DBD14046BDE8F0872DE9F0410446884627
:102D0000D4E90207C51BE168606816460844B5426D
:102D100006D94146FEF784FBB819E060BDE8F081B2
:102D20002A464146FEF77CFB761B08EB050132463E
:102D30006068FEF775FBE660F0E702E008C8121F66
:102D400008C1002AFAD170477047002001E001C194
:102D5000121F002AFBD170470121202803DA81408D
:102D60000548014003E0402802DA2038814009B1DB
:102D70000120704700207047FC06FFBD800701D08E
:102D8000002070470120704740680068401E0842DC
:102D900001D10120704700207047C3688B4206D8DC
:102DA00011440069491E814201D80120704700206A
:102DB0007047000030B585B00D46164C1621ADF8B1
:102DC00000101ECC0DF1040C8CE81E00124C0221E8
:102DD000012221706270A0700320E07021715920DF
:102DE0006071FE20A071694604F109007DDF0028B2
:102DF0000ED1BDF800002A46411CE1710921217263
:102E0000BDF808100844ADF8080001A9034872DFB6
:102E100005B030BDC0B80700A45E0020A85900204E
:102E200010B586B0062418220D496846FEF7F8FA58
:102E30000C480D49401AC008042101EB00400BA1C9
:102E400005F0A8F969462046FFF7B4FF002805D130
:102E50000A4C207874DF0121207873DF06B010BDA2
:102E6000D0B8070040CE070038CE07004164766531
:102E700072746973696E672E2E2E0000A8590020A7
:102E80002DE9F05FDFF89CB05C46DBF84890DBF89A
:102E9000246002F08FFF216B4718751A22482349DE
:102EA000401AC108042000EB0140804620A105F033
:102EB00071F9216B4944B94200D1002508232A4603
:102EC000384601F03DFD0700184817494FF0010A48
:102ED000A1EB00004FEAD0010AEB014404D02046E8
:102EE0001AA105F057F919E002F064FF00223146FB
:102EF00001F070F9DBF828200546D946AA4208D12E
:102F0000404619A105F046F9C9E9075AC9F8186001
:102F100004E020462B461A4905F047F93846BDE83B
:102F2000F09F00003C76002088CE070038CE0700D6
:102F3000456E746572206E72665F6466755F61705F
:102F4000705F636F6E74696E756500004661696CD1
:102F5000656420746F20636F7079206669726D7785
:102F60006172652E0000000053657474696E6720FD
:102F70006170702061732076616C696400000000EC
:102F8000F0BE070008B51346024600930648074BFB
:102F9000C01AC008012303EB00400B4604A105F052
:102FA0000CF906F0F5FA000088CE070038CE0700CD
:102FB00052656365697665642061206661756C742D
:102FC000212069643A203078253038782C207063CD
:102FD0003A203078253038782C20696E666F3A2098
:102FE0003078253038780000024606480649401AF5
:102FF000C008012101EB004004A105F0CFF806F064
:10300000C7FA000088CE070038CE07005265636516
:103010006976656420616E206572726F723A203045
:1030200078253038782100002DE9F04107461E4E02
:103030001E481F49326A401AC508012A04D00320DD
:1030400000EB05401BA12BE04FF44050184B174CF0
:103050004168E31A234A0220DB0800EB0344914253
:1030600006D1C1023B462048726B00F05DFF90B173
:1030700002F0A0FE01461C483B464130B26900F018
:1030800053FF58B1042000EB054018A105F082F869
:103090000120BDE8F081204618A101E0204626A1CC
:1030A00005F078F80020F4E73C76002088CE070091
:1030B00038CE0700426F6F742076616C696461746A
:1030C000696F6E206661696C65642E204E6F207694
:1030D000616C69642061707020746F20626F6F741E
:1030E0002E000000DBE5B1519C780020417070207B
:1030F00069732076616C696400000000426F6F7430
:103100002076616C69646174696F6E206661696CB8
:1031100065642E20536F6674446576696365206923
:10312000732070726573656E742062757420696EA9
:1031300076616C69642E0000426F6F742076616C5A
:1031400069646174696F6E206661696C65642E20C4
:1031500041707020697320696E76616C69642E001D
:103160002DE9F84F254C8146924660880E468142F3
:1031700041D800274FF6FF788DF80070684600F0C0
:1031800075F822786078A188884201DA401C00E056
:103190000020C0B2904204D19DF8000000F0B2F8C7
:1031A00027E065786078884201DA401C00E0002062
:1031B00060709DF8000000F0A5F8454519D0A068A2
:1031C000B9F1000F40F835A00DD066B16188E06814
:1031D000324605FB01004946FEF722F9A06800EBE4
:1031E000C500868002E000EBC50087800020BDE8B6
:1031F000F88F0420FBE70920F9E70000EC590020D4
:1032000010B50E4C03E0401C00E000202070207838
:103210006178814210D022786188E068A36802FB5F
:10322000010003EBC20153F83220898890472078CF
:10323000A1888842E9DAE6E710BD0000EC590020D9
:1032400030B5CB0008339DB293074FF0000401D096
:10325000072030BD044B9A602A44DA605C701C7011
:1032600058809980002030BDEC59002070B504468C
:1032700007F050F8012803D010A1432000F086F891
:10328000EFF3108172B61D4A9368012083B99060F4
:103290004FF0E020D0F88051194B1D401560C0F868
:1032A0008031D0F8843153604217C0F88421002067
:1032B0002070002900D162B670BD00002E2E5C2E59
:1032C0002E5C2E2E5C2E2E5C2E2E5C636F6D706F2E
:1032D0006E656E74735C6C69627261726965735C51
:1032E0007574696C5C6170705F7574696C5F706C2B
:1032F0006174666F726D2E6300000000B07D002067
:10330000FC06FFBD10B5044607F004F8012803D001
:103310000DA1512000F03AF81B498868002811D00F
:10332000002C0FD1EFF3108072B60B684FF0E02243
:10333000C2F800314B68C2F8043100228A600028CC
:1033400000D162B610BD00002E2E5C2E2E5C2E2EFB
:103350005C2E2E5C2E2E5C636F6D706F6E656E74CE
:10336000735C6C69627261726965735C7574696CB7
:103370005C6170705F7574696C5F706C6174666FAE
:10338000726D2E6300000000B07D00201CB56A46FF
:10339000CDE90001002144F20200FFF7F3FD1CBD5E
:1033A0002DE9F843274F274857F8246F846CB968F4
:1033B000AC2901D024B106E0406B0444361A02E087
:1033C00002F00CFD0446204820492346401A4FEAEB
:1033D000D008042101EB084005461D4A1DA10096B6
:1033E00004F0EBFEB868AC2806D13246A4F5804163
:1033F0001748FEF740F800B3324621461448FEF75E
:103400003AF8D0B128463346224620A104F0CDFE3A
:1034100004F050FD0028FBD102F0A0FA314620460E
:1034200003F0C4F8040005D0012101EB084023A1FA
:1034300004F0B0FE2046BDE8F8830024284626A10B
:10344000F6E700003C76002088CE070038CE070063
:1034500000100700566572696679696E6720424CF4
:103460003A20416464723A203078253038782C2034
:103470005372633A203078253038782C204C656EB2
:103480003A2030782530387800000000436F70799A
:10349000696E6720626F6F746C6F616465723A2049
:1034A0005372633A203078253038782C204C656E82
:1034B0003A20307825303878000000005265717568
:1034C00065737420746F20636F707920424C20669E
:1034D00061696C65640000004E6F20626F6F746CF0
:1034E0006F6164657220636F7079206E65656465D5
:1034F000642C20626F6F746C6F61646572207570EC
:103500006461746520636F6D706C6574652E000076
:1035100030B595B0040004D12E4940F24F40FFF77A
:1035200035FF2D494FF6FF702246488001208DF867
:1035300012004FF65960ADF8100004A90120A8DF71
:10354000002844D1254B0FCB8DE80F00A11C684605
:1035500062DF00283BD121491C2260390BA8FDF70E
:103560005FFF1F4D142205F1C401A8681290A078D6
:103570008DF84A002868139006A8FDF751FF12A89D
:10358000069013A807902088231D06AA0BA9AADF7E
:1035900000281CD11C2205F1D8010BA8FDF740FF23
:1035A000E8681290A0788DF84A0068681390142299
:1035B00005F1F40106A8FDF733FF12A8069013A841
:1035C0000790208804F10C0306AA0BA9AADF15B006
:1035D00030BD0000DCBF0700A859002098B90700E3
:1035E00090B80700F0B585B00D46040004D1374906
:1035F00040F28710FFF7CAFE25B934494FF4C47072
:10360000FFF7C4FE14216846FDF723FF207803234B
:1036100008280BD12E48C188491E89B2C1808288F2
:10362000002A4BD0002949D1C280237021786078CC
:1036300060228DF800208DF801108DF8020063786B
:103640000325012B16D0234823492278401AC008AD
:10365000022101EB004021A104F0A7FD60780B28B6
:1036600028D101F0ADF88DF80300002001F0B0F88A
:1036700004251FE0207809281CD2DFE800F01B1B7E
:103680001B211B1B051B2100D4E902706D46E91CA0
:10369000666807F01DFE044629193046C91C07F06C
:1036A00017FE044429193846C91C07F011FE2044AE
:1036B000C01CC5B22946684606F0F4FE05B0F0BD50
:1036C000D4E90112684606F0DCFEF1E7DCBF070032
:1036D000A859002040CE070038CE070044465520A8
:1036E00072657175657374202564206661696C6507
:1036F000642077697468206572726F723A2030783E
:10370000257800002DE9F0411D4C0026217AC907DB
:1037100033D01C49884230D01B481C49401AC1088C
:10372000042000EB0140054619A104F033FD608838
:10373000A0F57F41FF3916D028461DA104F02AFDCF
:10374000A068132140F00400A060608876DF0028A4
:1037500014D11B4CC8264FF47A47611C3846884761
:10376000761EFAD101E0207874DF05F0D1F806006A
:1037700003D1284613A104F00DFD3046BDE8F081C9
:10378000A859002020CE070040CE070038CE070001
:103790005368757474696E6720646F776E20424C4D
:1037A00045207472616E73706F72742E0000000099
:1037B000446973636F6E6E656374696E672E000093
:1037C000A0B80700424C45207472616E73706F722E
:1037D00074207368757420646F776E2E000000008B
:1037E00070B5204C06460020217AC90738D11E4802
:1037F0001E49401AC108042000EB014005461CA1E7
:1038000004F0C8FC2248E66001F012FD00F01CFB49
:10381000002825D103F0A0F838B11E4803F090F835
:10382000A06840F00200A06003E028461AA104F05E
:10383000B1FC01F019F8002812D116481C30FFF72E
:1038400067FE00280CD1FFF7EBFA002808D1A0682A
:1038500018A140F00100A060284604F09BFC002065
:1038600070BD0000A859002040CE070038CE0700E8
:10387000496E697469616C697A696E6720424C456A
:1038800020444655207472616E73706F727400002C
:10389000A8CE0700C45E00204E6F2061647665727A
:1038A000746973696E67206E616D6520666F756EF1
:1038B00064000000424C4520444655207472616EFD
:1038C00073706F727420696E697469616C697A656E
:1038D000642E00002DE9FE439F49A04B0122591A96
:1038E000C9080746051D02EB0148008804229C4ECA
:1038F0004FF0000902EB014421286ED037DC132879
:103900006CD01EDC01286AD0102854D0112868D051
:10391000122879D1204693A104F03CFCEA88204685
:103920009AA104F03BFCAA8820469EA104F036FC34
:103930002A892046A1A104F031FC6A892046A4A16D
:10394000ECE0142875D01A2874D01F285CD12046CA
:10395000A5A104F01FFC291D708875DF040053D059
:1039600040462246ACA104F019FC20461FE0512835
:103970007AD00EDC222878D0232868D024287BD067
:10398000502877D103B03946BDE8F043B04805F080
:103990008FBE5228D8D0552837D056286AD1B8794A
:1039A000002867D11321708876DF002862D0BDE837
:1039B000FE43FFF719BB2046A6A104F0EBFB2888C5
:1039C0007080F16809B101208847A549708875DFCA
:1039D00002004FD04046A3A1A0E07FE055E087E081
:1039E000FFE74FF6FF707080307A400704D4FFF78E
:1039F00017FA08B1FFF7F8FAF16800293AD003B0D6
:103A00000220BDE8F043084734E0FA88F72A14D2D0
:103A10009007B0F1404F0ED0D01F81B2481EC3179F
:103A200000EB937323F00303C01A081A801D85B2BC
:103A300004E078E081E0154600E0F72520462B46BB
:103A4000944904F0B2FB29467088B5DFADE7204603
:103A500091A104F09FFBCDF80090CDF80490B888B8
:103A60000022694690DF2DE046E02EE004E000BF32
:103A7000FFF7BAFABDE8FE836B89EA8803B02046F7
:103A8000BDE8F04391A104F090BB20469FA104F053
:103A900081FB734801AA163842F60521806A01901D
:103AA000CDF808D07088ADDF08B1FFF79DFA204649
:103AB000BDF800209FA104F071FB00231A46852168
:103AC00070887FDF0028D3D1D4E7287900906B7904
:103AD000AA792046A0A104F070FBCBE72046ADA157
:103AE00004F058FBCDF80090288869468FDFE9E79D
:103AF0000021708866DF58E7B8790028BAD03946C7
:103B0000534805F091FD0028B4D007F10801504852
:103B100005F0ACF90200ADD04046A9A103B0BDE864
:103B2000F04304F03BBB2046B2A104F033FB00217C
:103B30000A4628880B4686DF37E7002328881A467E
:103B40001946B1DF08B1FFF74FFA03B02046BDE8D0
:103B5000F043B2A104F01EBB38CE070040CE0700F0
:103B6000A8590020526563656976656420424C451A
:103B70005F4741505F4556545F434F4E4E5F504143
:103B800052414D5F55504441544500006D61785F8E
:103B9000636F6E6E5F696E74657276616C3A202534
:103BA000640000006D696E5F636F6E6E5F696E74B6
:103BB000657276616C3A202564000000736C617652
:103BC000655F6C6174656E63793A2025640000005E
:103BD000636F6E6E5F7375705F74696D656F75741A
:103BE0003A202564000000005265636569766564CB
:103BF00020424C455F4741505F4556545F434F4E0E
:103C00004E5F504152414D5F5550444154455F52C3
:103C100045515545535400004661696C75726520E5
:103C2000746F2075706461746520636F6E6E656378
:103C300074696F6E20706172616D65746572207257
:103C40006571756573743A2030782578000000003E
:103C5000E05E0020436F6E6E656374656400000073
:103C6000A6B807004661696C75726520746F20758F
:103C7000706461746520636F6E6E656374696F6EE6
:103C800020706172616D65746572733A20307825B9
:103C90007800000094BF070052656365697665642B
:103CA00020424C455F4741505F4556545F44415464
:103CB000415F4C454E4754485F5550444154455F21
:103CC000524551554553542E00000000526563651E
:103CD0006976656420424C455F4741505F455654C4
:103CE0005F444154415F4C454E4754485F555044F2
:103CF000415445202825752C206D61785F72785FCE
:103D000074696D65202575292E0000005265636574
:103D10006976656420424C455F4741505F45565483
:103D20005F5345435F504152414D535F524551559A
:103D3000455354004343434420666F7220736572B9
:103D400076696365206368616E67656420697320C6
:103D50003078253034780000526563656976656493
:103D600020424C455F4741505F4556545F5048598B
:103D70005F555044415445202852583A25642C2020
:103D800054583A25642C207374617475733A256411
:103D900029000000526563656976656420424C45E0
:103DA0005F4741505F4556545F5048595F555044F6
:103DB0004154455F524551554553542E0000000073
:103DC000436F756C64206E6F742068616E646C65FF
:103DD000206F6E5F6374726C5F70745F777269746A
:103DE000652E206572725F636F64653A20307825B6
:103DF00030347800526563656976656420424C45CD
:103E00005F4741505F4556545F5345435F494E46B7
:103E10004F5F5245515545535400000046696E6945
:103E2000736865642068616E646C696E6720636F97
:103E30006E6E2073656320757064617465000000A8
:103E4000007800F00100704738B50020009002F0C3
:103E5000B9FB00282DD117481749184A401AC10844
:103E6000042000EB0140044615A104F097F9134823
:103E700013DF00281DD1204619A104F08BF904F0AE
:103E800071FD002815D1684604F0D2FB002810D13E
:103E9000204619A104F07EF96946012004F0D2FB06
:103EA000002806D120461AA104F074F9684604F0EF
:103EB00061FC38BD40CE070038CE07000010070077
:103EC00053657474696E6720757020766563746FCE
:103ED00072207461626C653A203078253038780041
:103EE000456E61626C696E6720536F6674446576D7
:103EF0006963652E00000000436F6E666967757226
:103F0000696E6720424C4520737461636B2E00001C
:103F1000456E61626C696E672074686520424C452D
:103F200020737461636B2E0013B90378012B01D0E9
:103F300002F084BF012070470022C32100F51870F1
:103F400000F048B92DE9F043A1B00446DDE9289618
:103F500020200F46209098461546782102A8FDF7AC
:103F600078FA41212046FDF774FAB7F8940005EB82
:103F7000051107EB8101A84201D991F896602670DE
:103F8000320033D0012A0DD01B481C4D0123401BA9
:103F9000C00803EB0045022A0CD0032A20D0284693
:103FA00017A117E000224946404600F013F9C4F873
:103FB00001001BE020A9601CCDE900014B464246F0
:103FC000184902A801F0C8FD80B104F0FDFD0246C9
:103FD000284615A104F0E2F8002021B0BDE8F083E6
:103FE000B1F89820601C9A31FDF71AFA4A4641460A
:103FF000204602F023FFF0E768CE070038CE070026
:10400000496E76616C696420626F6F742076616CB2
:1040100069646174696F6E20747970653A202564F3
:1040200000000000B8B607006E72665F63727970B8
:10403000746F5F686173685F63616C63756C6174F2
:10404000652829206661696C656420776974682039
:104050006572726F722025730000000010B504466F
:104060000A480B49401AC008042101EB004009A18D
:1040700004F090F84FF0000034B10C490870BDE82E
:1040800010400B4802F094BC00F0E2FA88CE070022
:1040900038CE0700526573657474696E6720626F6D
:1040A0006F746C6F616465722E00000068590020A7
:1040B000514607002DE9F84F0546861C00208DF873
:1040C000000091460F464FF0010A6846FFF7CEF810
:1040D0001C4C60683860D4E901011B4F401A3968F4
:1040E000081A41F21C0104EB01080EE001214046D0
:1040F00000F0C9FF00F01EFE0146404600F0C3FF7D
:10410000D4E90101401A3968081A401C8642EDD8EA
:10411000B9F1000F03D0052065F3891002E00620F5
:1041200065F39F5061683A68114004EB8101C860F3
:104130006068304460609DF80000FFF7E3F8504687
:10414000BDE8F88F54810020145A002010B5436850
:104150009C18446021B905E013F8010B01F8010B2C
:10416000521EF9D2012010BD70B50D4604460A2931
:1041700002D10D21FFF7F8FFA0682268411CA16061
:104180001554D4E90101814204D32046BDE87040B2
:1041900003F0A0BA70BD0000044881684068814205
:1041A00001D1012070470020704700005481002099
:1041B00010B5040003D10549F020FFF7E7F80448E3
:1041C000C16B6160006CA06010BD0000DCC0070026
:1041D0003C760020F0B54FF0FF3622B11268D24392
:1041E00000230A4D0DE03246FAE7C45C6240082421
:1041F000D70700D037462F4087EA5202641EF7D116
:104200005B1C8B42F1D3D043F0BD00002083B8ED9E
:1042100010B504460068401C07D0204606F0A2FBFB
:104220002168814201D1012010BD002010BD000095
:1042300010B5104C90B06078002818D101F0F0FC57
:1042400018B10D49DB20FFF7A1F820220B49684681
:1042500001F006FD40236A4609490A4801F03CFC8A
:1042600018B10549E520FFF791F80120607010B002
:1042700010BD0000DC590020BCC4070068B6070070
:10428000E87C0020D0B60700F0B5146906468DB072
:1042900020681546271DE0B1022920D00A20009091
:1042A0006B4609AA304606F0BBF800280FD009A9D2
:1042B00001A8009A05F0E0FD01AE96E80F0005AEFA
:1042C00086E80F00236869683A4605A898470DB04C
:1042D000F0BD0DB03046BDE8F04005F041BE694686
:1042E000304605F0D3FD0028F1D0236869683A46CE
:1042F000684698470028EAD002980028F5D101982E
:1043000070600120E3E753689B7813F0C00303D08B
:10431000402B03D00020704700F002B8FFF7B4BF75
:104320002DE9FF410B465168064614468878334D07
:1043300000F00F0210F0300055F8225006D010287F
:1043400006D0202808D0302856D13EE022694DE022
:1043500061690120087047E0022B28D1042A26D881
:104360004FF0010869463046676905F08FFD002867
:104370001AD009E00B89226903FB00226846A8478E
:1043800070B13888401C3880029820B16168388844
:104390004A899042EED301987060029860BB02E0B7
:1043A0004FF00008F7E7404604B0BDE8F081D4E9DB
:1043B00004300F890288498907FB02338A421BD2E5
:1043C000521C02801A46616810E008886169072A59
:1043D000088009D1606801892069FDF73AF86068B2
:1043E0002169C06805F06DFD2269616804B030463E
:1043F000AC46BDE8F04160470020D5E758BD070056
:1044000038B51E4901200A68D20301D500040CE02A
:104410001B490A681523D2B2B3EBD20F07D10A6841
:10442000D20704D0086800F0560008600020FEF7AC
:10443000FBFD1449144A891AC908042202EB0144FD
:10444000B0B110200090684603F03CFCD0F8100595
:104450000099C84010F0010F0DD004F0CFF810F013
:10446000B10004D0204609A103F094FE012038BD1C
:1044700020460FA1F8E7204616A1F5E7000400400A
:104480002005004088CE070038CE0700444655205E
:104490006D6F6465207265717565737465642076EF
:1044A00069612047505245475245542E0000000094
:1044B000444655206D6F6465206265636175736560
:1044C00020617070206973206E6F742076616C6952
:1044D000642E0000444655206D6F6465207265713E
:1044E0007565737465642076696120627574746F94
:1044F0006E2E0000FEB519490446086808B1401E3A
:1045000008601748174AD4E90153801AC0080422EA
:1045100002EB004022789DB10E6821690296CDE938
:1045200000312B46012A16D00FA211A103F058FE2C
:104530006169002911D0E06803B0BDE8F040084788
:1045400009680091012A04D007A218A103F035FEE2
:10455000EEE720A2F9E71FA2E7E7FEBDC059002061
:1045600048CE070038CE0700657261736500000011
:10457000466C617368202573206661696C656420F0
:104580002830782578293A20616464723D25702CA2
:10459000206C656E3D307825782062797465732CC7
:1045A0002070656E64696E6720256400466C6173D7
:1045B0006820257320737563636573733A206164A3
:1045C00064723D25702C2070656E64696E672025CD
:1045D0006400000077726974650000007047000095
:1045E00010B50446801E062810D2DFE800F00D0347
:1045F000030F09090A494FF4701000F087FF05E026
:104600000120FFF72BFD01E002F05EFA054841684A
:10461000002903D02046BDE81040084710BD000027
:10462000B54A07006859002010B50446062801D095
:10463000072C02D1002002F043FB04480168002946
:1046400003D02046BDE81040084710BDA459002003
:1046500003F058FE03F02EFC0028FBD1BFF34F8F70
:1046600005480168054A01F4E06111430160BFF3A8
:104670004F8F00BFFDE700000CED00E00400FA05DD
:1046800010B50021024800F014FD80F3100010BDA9
:10469000709100202DE9FC4180461F4615460E46CC
:1046A00000240D4800F0ECFC38B11120BDE8FC817D
:1046B00006EB043003F050FF641CAC42F8D106480E
:1046C00000F0D5FCCDE900573346002202214046D8
:1046D00000F02AF80020E9E7FC5900202DE9F84312
:1046E000104D0F4680461E4691466946286800F0E8
:1046F00092FC040014D01C21FCF7ABFE01202071B9
:10470000C4F81490380BC4F80080C4E9026069460C
:10471000286800F0A1FC05F063FE0020BDE8F883E6
:104720000420FBE724BA07002DE9F04387B00446D4
:10473000DDE90E8980681D4616460F4600280BD01D
:1047400018216846FCF785FE02A88DF8007080E805
:104750006003A1686846884707B0BDE8F08330B5BC
:104760000446006887B00D46806800281FD01821D5
:104770006846FCF76EFE0195A0680590207910B19F
:10478000012810D107E001208DF800002069029077
:10479000E068039005E002208DF80000E068000367
:1047A000029060690490206881686846884707B075
:1047B00030BD0B2803D30B38C0B200F009B87047E6
:1047C0000249002208780A7070470000C45900208E
:1047D000014908700B207047C4590020014901208D
:1047E000087070476859002001490120087070471F
:1047F000A059002070B515460E46040004D10749A3
:104800004FF42C70FEF7C2FD2A46314604F17200C7
:10481000BDE87040012302F063BB0000BCC4070088
:1048200010B5040003D10E49DB20FEF7AFFD207860
:1048300018B90B49DC20FEF7A9FD94F85500094989
:1048400038B1012805D06068C968884205D90120BF
:1048500010BD606889688842F9D24FF0000010BD31
:1048600004C507003C7600203EB59DF8080020F006
:104870000F00401C20F0F00010308DF80800684652
:104880006DDF00282BD19DF80100401C8DF8010040
:1048900068466CDF002822D111481349007A82074C
:1048A0001048A0EB01004FEAD0004FF0040101EBEB
:1048B000004008D50D4C0EA1221DA36903F075FC24
:1048C000211DA06904E013A103F064FC19A10720D5
:1048D00082B202A87CDF002801D118487ADF3EBDF1
:1048E000A859002040CE070038CE0700C45E002043
:1048F00053657474696E6720616476206E616D65BE
:104900003A2025732C206C656E6774683A20256404
:10491000000000005573696E672064656661756C00
:1049200074206164766572746973696E67206E6164
:104930006D6500004466755461726700A6B8070093
:104940002DE9FC5F164607463A4A3B481D46101AB9
:1049500004224FEAD00902EB09408B468246B94255
:1049600005D136A103F016FC0020BDE8FC9F04D25F
:1049700036494FF04F00FEF709FD1DB9334950206D
:10498000FEF704FD2EB1380503D030495320FEF761
:10499000FDFCABEB0700040B03D12C495720FEF7BD
:1049A000F5FC0020009006F6FF704FEA103800F08A
:1049B000E9FFA54239D22C4637E0A04503D8354659
:1049C000CDF8048001E025030194002238460199C6
:1049D00001F07AFC0028C8D150463B465A461CA13B
:1049E000009503F0EAFB681E00F003002A1A00237A
:1049F00059463846D21C01F01DFD0028B5D1019959
:104A00001C48A8EB0108761B016B2F442944016365
:104A1000AB44002002F040F9009030B1012101EBDD
:104A2000094015A103F0B6FB01E0002EC5D10098A6
:104A30009BE7000088CE070038CE07004E6F20634A
:104A40006F7079206E65656465640000A0BE070024
:104A5000436F7079696E67203078257820746F20F5
:104A6000307825782C2073697A653A20307825785B
:104A7000000000003C7600204661696C656420748B
:104A80006F20777269746520696D61676520636F57
:104A90007079696E672070726F67726573732074C6
:104AA0006F2073657474696E677320706167652E1B
:104AB000000000000748084910B5401AC00803214B
:104AC00001EB004005A103F065FBBDE810400120AB
:104AD000FFF7C4BA88CE070038CE0700496E61637D
:104AE0007469766974792074696D656F75742E00C8
:104AF0000149416000207047F8B9070010B50B4923
:104B000041600B4800F0BCFA68B903F07DFF08492A
:104B10001C234FF4EE7208740448A1F5EE71001FD7
:104B2000006800F065FA002010BD000028BA0700F8
:104B3000A87F00202DE9FC5F0E008346DDE90C47CD
:104B4000C6F1000098469246814600D408460125E9
:104B500003E000BF90FBFAF06D1C5045FADAA8455F
:104B600000D9454624B1002E01DB780700D5641E2C
:104B7000B80702D5B8F1000F0AD0F80708D13CB148
:104B8000A54205D220215846641EFFF7EDFAF6E74C
:104B9000002E02DA4E462D2102E0780703D52B21A4
:104BA0005846FFF7E1FA07F0030002280BD1B8F1ED
:104BB000000F08D13CB1A54205D230215846641EF1
:104BC000FFF7D2FAF6E7CDE90047434652463146B1
:104BD000584606F09FFBBDE8FC9F02460020126885
:104BE000530713D502F00300012802D002280CD18C
:104BF00005E0C2F383100B68801C184404E0022314
:104C0000086803EB925210440860012070470000CE
:104C100002480068002800D001207047FC5900209D
:104C20000248007A002800D001207047A87F0020A9
:104C300038B54FF440521B49536800F500508B4281
:104C400004D044688C4201D1012400E000248B424E
:104C500026D143688B4223D11178142901D9526996
:104C600000E000221049B2FBF1F30278142A01D9C6
:104C7000406900E00020B0FBF1F0834203D0012442
:104C80000AA2009002E000240AA200900B480C49FE
:104C9000401AC008032101EB00400AA103F08DFA7D
:104CA000204638BDDBE5B15140420F006D616A6FAF
:104CB000720000006D696E6F7200000068CE070020
:104CC00038CE0700536F6674446576696365207556
:104CD0007064617465206973206120257320766596
:104CE0007273696F6E207570646174652E204375F0
:104CF0007272656E743A2025642E204E65773A20D4
:104D000025642E0070B5054608680C464A6886681A
:104D10002846314604F0F6FF6068286104F10C0073
:104D20006861B0780221B1EB901F01D1241D2C6184
:104D300070BD00002DE9FF410026274800F09DF9D5
:104D40002548001F074600F098F9244C2449A06824
:104D500000900D6800E000986946284004EB800050
:104D60000C30FFF73AFF0028F5D101AA009901EABB
:104D7000050304EB8303491CDB6842F82030401C28
:104D800000910228F2D3019800F0030001281AD004
:104D900002280ED013A14FF4C270FEF7F7FA38467E
:104DA00000F068F908B10098A06004B03046BDE892
:104DB000F0810198032101EB90500099BDF80A6041
:104DC00001EB900005E00198BDF80A60C0F3831084
:104DD00008440090E3E700006C910020548100201B
:104DE000145A00202E2E5C2E2E5C2E2E5C2E2E5C55
:104DF0002E2E5C636F6D706F6E656E74735C6C6984
:104E0000627261726965735C6C6F675C7372635C1C
:104E10006E72665F6C6F675F66726F6E74656E64EC
:104E20002E63000000F082FD4FF48051002000F05E
:104E30008DFBC8B91548C0F5FC2100F087FB98B977
:104E40000021134803F032FA03F01EF8114812490A
:104E5000401AC408032000EB044010A103F09AF9A3
:104E6000114800F08BFC08B1FEF7BEF803F022F801
:104E70000028FBD1012000EB04400CA103F08AF9CB
:104E800003F018F80028FBD1EEE70000001007003F
:104E90003555070088CE070038CE0700496E736984
:104EA0006465206D61696E00DD45070041667465CB
:104EB00072206D61696E2C2073686F756C64206E52
:104EC0006576657220626520726561636865642E2F
:104ED000000000002DE9F05F1E46DDF828B0914685
:104EE0008A46040003D124A1B620FEF74FFAB4F895
:104EF0000680607908FB00F8A8F10408464503D352
:104F00001DA1C420FEF742FAE788301DB0FBF7F17F
:104F1000B0FBF7F207FB1200D9F80050AA1942457E
:104F200001D9A8EB0605C9F8005001E02468491E24
:104F30000029FBD13E1A8846AE4215D817E000BFC3
:104F40002044001D0AEB0803BBF1000F324602D0DB
:104F50000146184600E01946FCF762FA0020246872
:104F6000AD1BB044AF4201D92E4600E03E46002DB5
:104F7000E6D1BDE8F09F00002E2E5C2E2E5C2E2E7A
:104F80005C2E2E5C2E2E5C636F6D706F6E656E7482
:104F9000735C6C69627261726965735C6D656D6F7B
:104FA000626A5C6E72665F6D656D6F626A2E630029
:104FB00030B5024651B103F08DF90021074C08E0ED
:104FC00034F821301568AB4202D11160002030BDA9
:104FD000491C8142F4D3052030BD000000000000D0
:104FE00010B5FCF762F908B1002010BD112010BD0A
:104FF00010B531B1B2FBF3F403FB14241CB109204A
:1050000010BD0E2010BD01600021416081608281D1
:10501000C381084610BD70B50C460546FCF7FAF88A
:10502000002802D021882868084470BD10B50A887D
:1050300049888A4203D1FCF72FF9012010BD0020D6
:1050400010BD70B50C460546FCF709F9002802D0E2
:1050500061882868084470BD10B50A8849888A426A
:1050600003D1FCF7F3F8012010BD002010BD002192
:1050700000F00FB8002100F012B8012100F01EB8B6
:10508000012100F011B808B56A46FCF75AF90098FA
:1050900008BD08B56A46FCF73AF9009808BD08B59E
:1050A0006A46FCF734F908BD08B56A46FCF722F9F0
:1050B00008BD08B56A46FCF711F908BD08B56A468F
:1050C000FCF718F9009808BD08B56A46FCF746F9E0
:1050D000009808BD38B5040004D115A14FF49270B2
:1050E000FEF754F900258DF800506846FEF7BEF82B
:1050F000206862680168914214D9491E01600D78E8
:105100001CB919A1E820FEF741F9208AE16805FBE6
:1051100000152068217A0278891A0279C9B28A4278
:1051200000D201719DF80000FEF7ECF8284638BD6A
:105130002E2E5C2E2E5C2E2E5C2E2E5C2E2E5C6374
:105140006F6D706F6E656E74735C6C6962726172A4
:105150006965735C62616C6C6F635C6E72665F62E2
:10516000616C6C6F632E63002E2E5C2E2E5C2E2ED7
:105170005C2E2E5C2E2E5C636F6D706F6E656E7490
:10518000735C6C69627261726965735C62616C6C9C
:105190006F635C6E72665F62616C6C6F632E63003E
:1051A00038B50C46050004D112A140F24710FEF7B5
:1051B000EDF824B90FA14FF4A470FEF7E7F8002032
:1051C0008DF800006846FEF751F81DB91749F52023
:1051D000FEF7DCF8E8682A68211A288AB1FBF0F1AA
:1051E0001068431C136001709DF80000FEF78AF8F8
:1051F00038BD00002E2E5C2E2E5C2E2E5C2E2E5CDA
:105200002E2E5C636F6D706F6E656E74735C6C696F
:10521000627261726965735C62616C6C6F635C6E13
:1052200072665F62616C6C6F632E63006851070089
:1052300010B5040002D0206830B901E00E2010BD86
:1052400019A1FF20FEF7A2F8606820B916A14FF45B
:105250008070FEF79BF8A06820B913A140F20110FE
:10526000FEF794F8E06820B90FA14FF48170FEF7C3
:105270008DF8208A20B90CA140F20310FEF786F8C1
:10528000207A61682268401AC0B2116004E0226886
:1052900011684B1C13600870401EC0B2F7D2216821
:1052A0000020087110BD00002E2E5C2E2E5C2E2ECC
:1052B0005C2E2E5C2E2E5C636F6D706F6E656E744F
:1052C000735C6C69627261726965735C62616C6C5B
:1052D0006F635C6E72665F62616C6C6F632E6300FD
:1052E0002DE9F041184819494FF48052401AC70877
:1052F000042000EB0745164615A1284602F04EFF94
:105300004FF0E024D4F8802128461FA104F5C07492
:1053100002F044FF60172060C4F800016060C4F828
:10532000040101F05BF928B1012000EB074021A145
:1053300002F030FF02F0BEFD0028FBD13046BDE890
:10534000F04100F053B8000088CE070038CE0700C7
:1053500052756E6E696E67206E72665F626F6F74F3
:105360006C6F616465725F6170705F737461727499
:10537000207769746820616464726573733A2030C1
:10538000782530387800000044697361626C696E7A
:105390006720696E74657272757074732E204E5634
:1053A00049432D3E494345525B305D3A20307825D4
:1053B000780000004661696C65642072756E6E69E4
:1053C0006E67206E72665F6466755F6D62725F699C
:1053D00072715F666F72776172645F616464726537
:1053E00073735F73657428290000000070B506466A
:1053F0002648C0F5FE2100F0A9F8040024482549FC
:10540000A0EB01004FEAD0004FF0010101EB004595
:1054100007D02846224620A102F0C0FE2046FDF714
:10542000E3FD00F0C7FC014629488069421EC2F333
:105430000B02801A0144002001F6FF7100F086F88B
:10544000040004D02846224622A102F0A7FE201E16
:1054500001D0FDF7C9FDEFF30580C105D6E9004590
:10546000C90D4FF0000080F3148880F3108880F39A
:10547000118880F3138803D023495820FDF786FF55
:1054800084F30888AC46BDE8704060470010070010
:1054900088CE070038CE0700436F756C64206E6FAE
:1054A000742070726F7465637420626F6F746C6FB8
:1054B0006164657220616E642073657474696E67DF
:1054C000732070616765732C20307825782E00007A
:1054D0003C760020436F756C64206E6F7420707290
:1054E0006F7465637420536F667444657669636591
:1054F00020616E64206170706C69636174696F6EA5
:105500002C20307825782E0004BE070070B5084D99
:1055100004460E46686805F0B5FE002C06D03246FB
:1055200021466868BDE8704005F09EBE70BD000071
:10553000705900200348D0F804050349097B00EBAB
:10554000016070470040024070590020F0B50A0524
:1055500002D1B0F5FE2F01D90720F0BD134D000B8D
:10556000491E124F01222E1D103700EB113407F196
:10557000040C17E04309C3F1000100EB411E02FADD
:105580000EF106D0012B06D0022B06D0032B08D13A
:1055900005E0296005E0316003E0396001E0CCF806
:1055A0000010401CA042E5D90020F0BD00060040DC
:1055B0002DE9F0413A483B49384E401AC5080420CD
:1055C00000EB05400027044637A102F0E3FDB06878
:1055D00001280ED0A52813D0AA2818D0AC281ED098
:1055E000032000EB054039A102F0D4FD0020BDE806
:1055F000F08120463CA102F0CDFDFDF741FC0CE01E
:1056000020463CA102F0C6FD04F06AFF0DE02046F2
:105610003BA102F0BFFDFDF7C3FE024607E02046B6
:105620003AA102F0B7FD05F029F8024601271D490D
:105630001B4B0120591AC90800EB014522B128462D
:1056400036A1B36802F0B1FD304600F0D7FBDFF8B9
:105650000081002188F800103E4801F01DFB06463D
:1056600098F8000020B93C4940F2A510FDF78EFEE5
:105670002EB1284639A102F08DFD0320B7E70120A5
:10568000002FB4D005492439096A0129AFD1204639
:10569000394902F07FFD0220A9E700006076002072
:1056A00088CE070038CE0700456E746572206E7292
:1056B000665F626F6F746C6F616465725F66775F5F
:1056C0006163746976617465000000004E6F206646
:1056D00069726D7761726520746F20616374697699
:1056E0006174652E0000000056616C696420417091
:1056F0007000000056616C69642053440000000093
:1057000056616C696420424C0000000056616C696F
:1057100064205344202B20424C00000041637469F4
:10572000766174696F6E206661696C656420776963
:105730007468206572726F72202564202862616E21
:105740006B20636F64653A2030782578290000006B
:10575000A0590020E9470700A0BE0700436F756C01
:1057600064206E6F74207772697465207365747439
:10577000696E67732E00000038BF07002DE9F843FB
:10578000044644484449401AC108042000EB014043
:10579000054642A102F0FEFC464F10207C600090BE
:1057A000684602F08FFA009A434900EB82004FF0FE
:1057B0000008C0F80017404601F000F9002852D157
:1057C000FFF7F6FE344A334B01219A1AD20801EB57
:1057D000024420B1012828D0022844D105E04FF42A
:1057E0007016FEF70DFE10B93AE04FF4A02600F057
:1057F000C9F8324A20211820FDF722FD08B1FDF733
:10580000F3FB02F0FBFE1621B1EBD00F09D102F041
:10581000F5FEC00705D002F0F1FE294920F0B100E5
:10582000086000F0A3FEF0B903E00120FEF716FCCB
:105830002AE024493046FFF769FE234800F04AFE7B
:1058400088B9284621A102F0A5FC00BF00F086F827
:10585000FDF7D6FC02F02EFB0028F7D141DFF5E77B
:1058600001F032F810B10320BDE8F88387F800801A
:105870001A4801F09DF8387820B919A14FF4027048
:10588000FDF784FDFFF72CFD204625A102F082FCE8
:10589000E9E7000088CE070038CE0700496E206E89
:1058A00072665F626F6F746C6F616465725F696E60
:1058B00069740000685900200C000300845A00201D
:1058C0001C050040B54A0700E1450700456E7465B8
:1058D00072206D61696E206C6F6F7000DD4707008C
:1058E0002E2E5C2E2E5C2E2E5C2E2E5C2E2E5C63BD
:1058F0006F6D706F6E656E74735C6C6962726172ED
:105900006965735C626F6F746C6F616465725C6E05
:1059100072665F626F6F746C6F616465722E630094
:10592000556E726561636861626C650010B540F622
:10593000F8700168491C02D1074902F025FE40F6C3
:10594000FC700168491C05D1BDE810404FF4FC21F2
:1059500002F01ABE10BD00000010070010B503F0E1
:1059600083F9002803D0BDE8104005F0EDBD10BD5F
:10597000034A93680A4601469860184605F074BCCD
:10598000705900202DE9F0411A4E307800282ED1B0
:1059900003F06AF91849194A0127891AC90803222C
:1059A00002EB014500281DD0154804682846224610
:1059B00014A102F0F3FBA4F54864962C00DC9624B5
:1059C00005F0C2FD2846224615A102F0E7FB214959
:1059D0002046FFF7CDFF4FF0E0214FF48030C1F8B3
:1059E000000103E028461CA102F0D4FB3770BDE89B
:1059F000F0810000A159002038CE070038CE070002
:105A00000405014057445420656E61626C65642052
:105A10004352563A2564207469636B73000000009A
:105A20005374617274696E6720612074696D657268
:105A300020282564207469636B732920666F7220A7
:105A400066656564696E67207761746368646F6713
:105A50002E00000085B50700574454206973206E5E
:105A60006F7420656E61626C6564000040688068D8
:105A7000004710B542680830527900F0F1F8002074
:105A800010BD2DE9F04399B01C4690460D460846DE
:105A9000DDF88090FFF7EAFF6E6807467079A04254
:105AA00000D804462246414611A800F015F9727943
:105AB000494601A800F0D4F801AB224611A905F12E
:105AC00008000097FBF77CFE18B1002019B0BDE874
:105AD000F08348F24250F9E770B516460C46054689
:105AE00000F0E2F800280ED1AA791946304600F0FD
:105AF000E8F8002807D131462046FFF7BAFF002812
:105B000001D10149216070BD7052464D2DE9F84325
:105B10000C46DDE908578146984616460D49204651
:105B200000F0B6F8002810D160683946407942008C
:105B3000284600F0C6F8002807D146B14346324651
:105B4000214648460095FFF79CFFBDE8F88348F2E0
:105B50001050FAE77052464D2DE9F0411D46DDE93F
:105B600006871646044600F02DF800280DD12A4677
:105B70003146204600F03CF8002806D13A4641461E
:105B80002046BDE8F04100F002B8BDE8F08170B5F4
:105B900015460E46044605F0C7FC002807D13EB165
:105BA00060682968C268914205D248F2145070BDFD
:105BB00048F2135070BD83682A4631462046BDE83E
:105BC0007040184710B550B161B141600968044692
:105BD0008847002802D105482060002010BD48F207
:105BE000015010BD48F2105010BD00006E524648E2
:105BF00070B515460E46044605F096FC00280BD1FC
:105C000046B155B160682A46314643682046BDE832
:105C10007040184748F2105070BD002070BD000061
:105C20002DE9F0410B480C4D0C4F401BC6080120DC
:105C30003870002406E000BF55F834008047002883
:105C400005D1641CB442F7D3022038700020BDE8AF
:105C5000F08100000000000000000000A2590020B8
:105C600070B514460D46064600F036F8291930196D
:105C70002246BDE8704000F02FB870B50C460546CE
:105C800000F064F828192146BDE8704000F05EB8C5
:105C900028B10068884205D048F24050704748F269
:105CA000105070470020704728B139B10022C1E977
:105CB00000201046704748F21050704748F21350C9
:105CC000704720B1914205D048F21150704748F218
:105CD000105070470020704770B516460C460500FE
:105CE00003D10AA14520FDF751FB1CB907A14620AD
:105CF000FDF74CFBA919491E04E000BF14F8010B85
:105D000001F80109A942F9D270BD00002E2E5C2EC7
:105D10002E5C2E2E5C2E2E5C2E2E5C636F6D706FB3
:105D20006E656E74735C6C69627261726965735CD6
:105D300063727970746F5C6E72665F63727970748F
:105D40006F5F7368617265642E63000070B50D4605
:105D5000040003D107A13320FDF718FB6019401E92
:105D600005E02178027804F8012B00F80119A0421F
:105D7000F7D270BD2E2E5C2E2E5C2E2E5C2E2E5C4D
:105D80002E2E5C636F6D706F6E656E74735C6C69E4
:105D9000627261726965735C63727970746F5C6E54
:105DA00072665F63727970746F5F73686172656445
:105DB0002E6300004FF44050074A4168914207D1DA
:105DC0008068411EC1F30B01401A00F6FF70704756
:105DD0004FF4805070470000DBE5B15100B5FFF78C
:105DE000E9FF054989690A18401E0844C0F30B0001
:105DF000101A00F6FF7000BD3C7600200021016003
:105E00004160816001480163704700003C760020DA
:105E10002DE9FF4F8B466948694981B0401AC10896
:105E2000042000EB0144009166A1204602F0B2F983
:105E300020466CA1019A02F0B1F9BBF1000F01D02C
:105E40006EA200E06FA2204670A102F0A7F90398AD
:105E500008B16AA200E06BA2204671A102F09EF98F
:105E6000049808B165A200E066A2204670A102F085
:105E700095F94FF4405041687348814201D15FA2C7
:105E800000E060A2204671A102F088F9204673A1CB
:105E900002F080F9754D204675A1AB692A6A02F0BF
:105EA00084F920467AA16B6AEA6A02F07EF94FF023
:105EB0000009DFF8FCA10CE0012650B1012812D046
:105EC000B9F1020F1ED07B49AC20FDF75FFA00202C
:105ED0001AE0FFF783FF8046039888B16348006AA1
:105EE00001280BD00CE0FFF765FF8046049828B925
:105EF0004FF4405041685448814201D0012604E0EB
:105F0000002602E04FF480508046D04503D969490D
:105F1000B120FDF73BFA68490198A1EB0801A1F512
:105F20000041814201D2012700E0002747EA0B052A
:105F300020464A4661A102F031F92046424662A15C
:105F400002F02CF90FB12DA200E02EA2204664A190
:105F500002F024F90EB129A200E02AA2204666A18F
:105F600002F01CF90DB125A200E026A2204667A18F
:105F700002F014F9B54308D0B9F1020F05D209F1C6
:105F80000100C0B28146022896D957B1009802217B
:105F900001EB004062A102F0FDF8042005B0BDE86D
:105FA000F08FB9F1000F07D0204668A102F0F2F897
:105FB0002E481830FFF722FF0020EFE788CE0700B9
:105FC00038CE0700456E746572206E72665F646637
:105FD000755F63616368655F707265706172652883
:105FE0002900000072657175697265645F73697A72
:105FF000653A20307825782E0000000074727565AF
:106000000000000066616C736500000073696E67D4
:106010006C655F62616E6B3A2025732E0000000094
:106020006B6565705F6170703A2025732E0000000B
:106030006B6565705F736F66746465766963653AF6
:106040002025732E00000000DBE5B15153445F5062
:10605000524553454E543A2025732E0042616E6BD3
:1060600020636F6E74656E74733A00003C76002096
:1060700042616E6B203020636F64653A2030782572
:106080003032783A2053697A653A203078257800A2
:1060900042616E6B203120636F64653A2030782551
:1060A0003032783A2053697A653A20307825780082
:1060B000009006007CC20700001007007061737337
:1060C0003A2025642E00000063616368655F6164A7
:1060D00064726573733A20307825782E00000000D2
:1060E00063616368655F746F6F5F736D616C6C3A59
:1060F0002025732E000000006B6565705F66697275
:106100006D776172653A2025732E000064656C65B9
:1061100074655F6D6F72653A2025732E0000000074
:1061200041626F7274696E672E2043616E6E6F7488
:1061300020666974206E6577206669726D7761727A
:1061400065206F6E2064657669636500496E7661CF
:106150006C69646174696E67206170702E00000064
:1061600070B50C46050004D121494FF4AC70FDF721
:106170000DF924B91E4940F25910FDF707F91D48E1
:106180001D4B2978C01A0422C00802EB00400929DF
:1061900027D2DFE801F02605260B15261B260F0067
:1061A00021462846BDE8704002F066BD13A101F00B
:1061B000F1FF11E021462846BDE8704002F000BE24
:1061C00021462846BDE8704002F098BD14A101F0B8
:1061D000E1FF4FF40070E0602046BDE87040FDF73D
:1061E000E7BFBDE8704002494FF4BC70FDF7CEB880
:1061F000DCC0070050CE070038CE070048616E644F
:106200006C65204E52465F4446555F4F505F435287
:10621000435F4745542028636F6D6D616E642900AC
:1062200048616E646C65204E52465F4446555F4F30
:10623000505F4F424A4543545F53454C45435420B9
:1062400028636F6D6D616E642900000070B50E46A5
:10625000040004D11B4940F27520FDF797F826B9D8
:10626000184940F27620FDF791F820780125092899
:1062700020D2DFE800F01F051F0F141F1A1F0A00AD
:106280003146204602F080FE19E03146204603F0F8
:10629000D1F814E03146204602F038FE0FE03146D6
:1062A000204602F07BFF054609E03146204603F018
:1062B00075F804E0034940F29720FDF767F8284697
:1062C00070BD0000DCC007002DE9F843134C074601
:1062D0000D4620680090124812499046401AC608A0
:1062E000042000EB06402B463A460FA101F065FF63
:1062F00043462A4639461C4801F040FB050009D0B8
:10630000022000EB06402A4618A101F047FF28466C
:10631000BDE8F8832068401C2060F8E7C0590020E1
:1063200048CE070038CE07006E72665F6673746FE2
:10633000726167655F657261736528616464723D4F
:10634000307825702C206C656E3D25642070616767
:106350006573292C20717565756520757361676596
:106360003A20256400000000705A00206E72665FBB
:106370006673746F726167655F6572617365282902
:10638000206661696C656420776974682065727243
:106390006F7220307825782E000000000C490D4ADD
:1063A00010B5891AC908042202EB014200281046E0
:1063B00004D009A101F0EEFE114903E011A101F0A2
:1063C000E9FE1A49BDE810400022194801F036BB29
:1063D00048CE070038CE0700496E697469616C6960
:1063E0007A696E67206E72665F6673746F7261673A
:1063F000655F7364206261636B656E642E000000EC
:1064000034BA0700496E697469616C697A696E67AC
:10641000206E72665F6673746F726167655F6E7619
:106420006D63206261636B656E642E0004BA0700C1
:10643000705A00202DE9FC47154C80460F46206815
:106440001549CDE9002013489946401AC60815465B
:10645000042000EB06403B464246104901F0B6FEE0
:106460002B463A4641460E48CDF8009001F0AEFB6F
:10647000050009D0022000EB06402A4609A101F0E0
:106480008DFE2846BDE8FC872068401C2060F8E7A8
:10649000C059002048CE070038CE070024C00700AE
:1064A000705A00206E72665F6673746F7261676502
:1064B0005F77726974652829206661696C6564205C
:1064C00077697468206572726F7220307825782E33
:1064D0000000000070B51149086011481149401AC8
:1064E000C508032000EB05400FA101F053FE00207A
:1064F000FEF79AF8114800F041FC040008D0012092
:1065000000EB054022460EA101F048FE204670BD7A
:10651000BDE87040094800F0A7B80000A459002069
:1065200088CE070038CE0700456E746572696E67C5
:1065300020444655206D6F64652E000029460700F3
:10654000436F756C64206E6F7420696E6974616C42
:10655000697A6520444655207472616E73706F725B
:10656000743A203078253038780000000648074912
:1065700010B5401AC008042101EB004004A101F04D
:1065800009FE002010BD000088CE070038CE0700AD
:10659000696E207765616B206E72665F6466755FF9
:1065A000696E69745F757365720000001FB58908B4
:1065B000002201AB009283E80700684618DF04B0B0
:1065C00010BD00001FB5044B0FCB8DE80F006846CF
:1065D00018DF04B010BD0000A8B907004FF48050C8
:1065E000410408600020704770B50E460178134CD6
:1065F000062901D0012901D1017C217021780125D2
:10660000012911D0022913D00D480E49401AC008A3
:10661000012101EB00400CA101F0BCFD0020207025
:1066200005207070284670BD3146FFF799FDF9E7E7
:106630003146FFF70BFE0546F4E70000C85900207D
:1066400050CE070038CE0700496E76616C69642031
:106650006F626A656374207479706520696E207258
:106660006571756573742E0010B5040011D001209A
:10667000FFF794FE00280BD100F0EEFC00F0CEFDF9
:1066800048B10949081F00F057FD012803D0032035
:1066900010BD072010BD04480838C4600020FEF774
:1066A00097F8002010BD0000D059002010B5816877
:1066B00089B10A4A1821FCF753FD040009D00848A3
:1066C0000849401AC008022101EB004006A101F070
:1066D00061FD204610BD072010BD000005670700C2
:1066E00050CE070038CE07005363686564756C654B
:1066F000722072616E206F7574206F6620737061F6
:1067000063652100AFF3008070B50546806886B0F0
:1067100020B9284940F2CF20FCF738FE182226493C
:106720006846FAF77DFE28788DF800002348244B50
:106730002A78181A0421C008224E01EB00440D2AC1
:106740001CD2DFE802F01B140714141B141B141BCB
:106750001B1B0C0020461CA101F01CFD17E020466D
:1067600022A101F017FDF168072088470FE0694674
:106770002846FFF739FF50B906B070BD032101EB81
:10678000004020A101F00AFD02208DF801009DF8D3
:106790000120204623A101F001FDD5E90112684640
:1067A00090479DF801000128E6D0F1680520884750
:1067B000E2E70000DCC00700D0B9070038CE0700D0
:1067C00050CE0700C859002048616E646C65204EA9
:1067D00052465F4446555F4F505F524543454950CE
:1067E000545F4E4F5449465F5345540048616E64B0
:1067F0006C65204E52465F4446555F4F505F4142A4
:106800004F525400496E76616C6964206F70636FFB
:1068100064652072656365697665643A2030782521
:10682000782E0000526571756573742068616E641E
:106830006C696E6720636F6D706C6574652E205295
:106840006573756C743A20307825780038B1054945
:1068500001600549416001210172002070470E204E
:10686000704700006D680700A568070010B50C00B0
:1068700001464FF0110007D02278052A05D2DFE843
:1068800002F00F050D0F0F000E2010BD084600F09E
:1068900073F80028F9D10221217010BD112010BD1C
:1068A000082010BD0246082041B10B78022B04D10C
:1068B000022A05D0032A00D1112070470E2070470C
:1068C000002003220A70704770B510480024D0F8E9
:1068D0002413491C03D1D0F86403401C13D00C4886
:1068E0000C49401AC008042101EB00400AA101F044
:1068F00051FC4FF4FE25284601F02EFEC922034923
:10690000284601F059FE204670BD00003C7600206C
:1069100060CE070038CE070045726173696E67204C
:1069200073657474696E6773207061676520616454
:10693000646974696F6E616C20646174612E00001B
:1069400010B528B11C220349FAF76AFD002010BDDA
:106950000E2010BD64F3070010B5064C002218216C
:10696000201DFDF737FC2168814201D1012010BDB7
:10697000002010BD64F3070070B50C4D0400D5F87D
:10698000640305F5597503D0401C03D0082070BD81
:106990000E2070BD00221821201DFDF71BFC206079
:1069A00007222146284629DF70BD000000F00700BD
:1069B000014903F06BBF000000F0070070B5054609
:1069C00012481349401AC408042000EB044011A1E6
:1069D00001F0E0FB2846FFF7E1FC02004FF0010068
:1069E00000EB044402D0204613A108E000F06CF84C
:1069F000002000F051F9020005D0204619A101F055
:106A0000CDFB032070BD002070BD000058CE0700F4
:106A100038CE070043616C6C696E67206E72665FEA
:106A20006466755F73657474696E67735F696E69B8
:106A30007428292E2E2E00006E72665F6466755FC4
:106A4000666C6173685F696E697428292066616984
:106A50006C65642077697468206572726F723A2081
:106A6000257800006E72665F6466755F7365747486
:106A7000696E67735F77726974655F616E645F6288
:106A800061636B75702829206661696C6564207785
:106A9000697468206572726F723A20257800000070
:106AA00010B5FF224FF400710648FAF7CBFC0548F9
:106AB00020212438FAF7CDFC024900205C39086314
:106AC00010BD0000987600202DE9F05F4048FDF7EA
:106AD0009FFB404E074634682046FDF799FB4FF078
:106AE000000A58B16068012806D02046FDF724FA54
:106AF000D4F85C12884201D1012400E00024364819
:106B00003649DFF8DC80401AC00803214FF0020943
:106B10004FF4607B01EB0045F7B1042101EB00402D
:106B2000074630A101F036FB5A4629494046FAF79C
:106B300077FCDCB1384631A101F02CFB36684446C5
:106B40005422311D201DFAF76BFC4FF4327206F10E
:106B50005C0104F15C0007E06CB32846324901F0A7
:106B600019FB5A461E483168FAF75AFCD8F8040057
:106B7000444601281DD128462CA101F00BFB3649C3
:106B8000402201F5E470FAF74BFC33491C224031F6
:106B900001F5E470FAF744FC84F860A2012184F85E
:106BA000A1122E4884F8E2A2E169C0F82210C4F8CC
:106BB0000490BDE8F09F4C4609EB0040284901F0E5
:106BC000E9FA59460648FAF744FCC8F80440F0E7E9
:106BD00000F00700D859002058CE070038CE070033
:106BE0003C7600205573696E672073657474696E16
:106BF000677320706167652E00000000436F707935
:106C0000696E6720666F7262696464656E20706188
:106C10007274732066726F6D206261636B75702091
:106C2000706167652E0000008CC107004F6C642006
:106C300073657474696E677320706167652064653D
:106C40007465637465642E20557067726164696E43
:106C50006720696E666F2E0098770020BC78002050
:106C600028C1070070B50546094803F07BFE084CB3
:106C700020602046FDF760F9C4F85C02A4F5E063EB
:106C80002A462146BDE87040024803F071BE00006C
:106C90003C76002000F0070070B505460020FFF7A5
:106CA000E1FF040003D10349284603F0EFFD20462D
:106CB00070BD00003C7600204FF48050704700000B
:106CC0002DE9F0471449DFF854808146A1EB080014
:106CD000C708134813490026401AC108042000EBD6
:106CE000014005463A4610A101F058FA00240EE092
:106CF00008EBC400416848468847060006D028468D
:106D00003346224612A101F050FA02E0641CBC4254
:106D1000EED33046BDE8F08728CE070020CE07002E
:106D200088CE070038CE07005368757474696E67A3
:106D300020646F776E207472616E73706F727473FB
:106D40002028666F756E643A2025642900000000D3
:106D50004661696C656420746F2073687574646F34
:106D6000776E207472616E73706F72742025642C5C
:106D7000206572726F722025640000002DE9F047D3
:106D80001449DFF854808146A1EB0800C708134876
:106D900013490026401AC108042000EB01400546B3
:106DA0003A4610A101F0FAF900240DE058F8341029
:106DB00048468847060006D028463346224612A198
:106DC00001F0F3F902E0641CBC42EFD33046BDE8A9
:106DD000F087000028CE070020CE070088CE0700ED
:106DE00038CE0700496E697469616C697A696E67AB
:106DF000207472616E73706F7274732028666F7581
:106E00006E643A20256429004661696C65642074CB
:106E10006F20696E697469616C697A65207472614A
:106E20006E73706F72742025642C206572726F729D
:106E300020256400012203F0DFB8000038B51446B5
:106E400002780B46FAB1012A09D0022A1DD0032A82
:106E500023D0174940F2D930FCF798FA25E0D0F852
:106E60000150002221461846FDF7B4F9A8420AD085
:106E7000104811490122401AC008042101EB0040CA
:106E80000EA101F08BF9012038BD01B02246BDE80A
:106E900030400023401C00F023B8411C4022002059
:106EA000009400F017FA0128EED0002038BD000051
:106EB000BCC4070068CE070038CE07004352432009
:106EC000636865636B206F6620617070206661691E
:106ED0006C65642E2052657475726E202564000006
:106EE0002DE9F043A9B007462020894628901C468A
:106EF00090460125782102A8FAF7ABFAFDF798F938
:106F00002CB12022394620A8FEF7E6FE20AF244807
:106F100024494346401AC608042000EB06400446B4
:106F20004A4621A101F041F928A92C48CDE90001E8
:106F300043464A462A4902A8FEF70EFE020006D042
:106F4000012000EB064027A101F028F922E02022D1
:106F500039462248FAF78FFAE8B1022000EB0640E2
:106F60002DA101F017F9204632A101F013F92046B6
:106F70002022394601F0BAF8204633A101F00AF97F
:106F800020462022154901F0B1F800BF00F092FF21
:106F90000028FBD1002529B02846BDE8F083000079
:106FA00068CE070038CE07004861736820766572A6
:106FB000696669636174696F6E2E2073746172749F
:106FC00020616464726573733A20307825782C20D0
:106FD00073697A653A20307825780000907D00202A
:106FE000B8B60700436F756C64206E6F74207275BD
:106FF0006E20686173682076657269666963617482
:10700000696F6E20286572725F636F6465203078E7
:107010002578292E0000000048617368207665728B
:10702000696669636174696F6E206661696C656425
:107030002E00000045787065637465642046572013
:10704000686173683A00000041637475616C2046A2
:107050005720686173683A0010B50648064C806B8B
:1070600020B103F0A3FF08B1012000E00020207050
:1070700010BD00003C760020DC5900202DE9F041D5
:10708000144C07460D46E06BA26B01264119914254
:107090000BD911481149401AC008012101EB0040E9
:1070A0000FA101F077F8032610E00A492A465C3167
:1070B00008443946FAF7B4F9E06B064A2844E0631D
:1070C000403229463846FDF785F820643046BDE851
:1070D000F08100003C76002068CE070038CE070023
:1070E000496E697420636F6D6D616E64206C6172AE
:1070F000676572207468616E206578706563746579
:10710000642E000070B504004FF0010504D0B4F502
:10711000007F03D9042508E0032506E00449002088
:107120000870FFF7BDFC03488463284670BD00006B
:10713000DC5900203C7600202DE9F0410646244829
:107140000F46254BD0E90E1222484FF00108C01A15
:10715000C00808EB00448A4205D020461FA101F078
:1071600019F8082430E0244D287840B1FEF736FEA7
:1071700030603946E86804F06BF9044624E003F017
:1071800015FFE0B100F050F8044600203060386090
:10719000012C0ED13946E86804F05AF9044601285A
:1071A00007D132463968E86804F00EF90446012830
:1071B00002D0FFF775FC07E085F8008004E0204668
:1071C0000EA100F0E7FF05242046BDE8F081000095
:1071D0003C76002068CE070038CE0700457865630E
:1071E0007574652077697468206661756C747920A0
:1071F0006F66667365740000DC5900204661696C37
:10720000656420746F206465636F646520696E69CE
:1072100074207061636B65740000000001480078A1
:1072200070470000DC590020F8B51C4C251D0020DB
:1072300094F86C31014602463BB194F8D802B4F898
:10724000DA2204F5B87504F53771154CA36800937C
:10725000636800F03FF80646012805D1281D00F0BC
:1072600043F90646012816D00E480F49401AC508B2
:10727000022000EB05400DA100F08CFF042000EB84
:10728000054510A1284600F085FF2089616882B27B
:10729000284600F02BFF3046F8BD0000BC790020E6
:1072A000DC59002068CE070038CE070050726576A2
:1072B000616C69646174696F6E206661696C656494
:1072C0002E000000496E697420636F6D6D616E64FD
:1072D0003A0000002DE9F047A2B080462020DDF8FA
:1072E000A8900F4620909A461646782102A8FAF7F1
:1072F000B0F800202190FCF79BFF40484049401A1D
:10730000C508032000EB054004463EA100F042FF03
:1073100057B1B8F1000F20460ED044A100F03AFF5B
:10732000162022B0BDE8F087022000EB054045A101
:1073300000F030FF1320F4E74A4647A100F02EFF8B
:1073400020A94C48CDE900014B4652464A4902A8C3
:10735000FEF702FC08B9402E01D00A20E1E74548BB
:10736000324639464038FAF75BF8204643A100F030
:1073700011FF404820214038FEF77FFC3D48402166
:107380004038CDE90001A0F148013A4A21A8209BEC
:10739000FEF7BCFB02002BD0012000EB05403CA116
:1073A00000F0FCFE042000EB054442A1204600F062
:1073B000F1FE304920464022403900F097FE204639
:1073C0003FA100F0E7FE20982A4982B2204600F053
:1073D0008DFE20463CA100F0DDFE204640223D49C6
:1073E00000F084FE00F066FD0028FBD1052098E740
:1073F000204639A100F0CEFE012092E768CE0700BA
:1074000038CE07005369676E6174757265207265C6
:107410007175697265642E20436865636B696E6778
:10742000207369676E61747572652E00496E7661AE
:107430006C6964207369676E617475726520747914
:10744000706500004E6F207369676E6174757265B8
:1074500020666F756E642E0043616C63756C617499
:10746000696E67206861736820286C656E3A202514
:1074700064290000707D0020B8B607005665726967
:107480006679207369676E6174757265000000002B
:107490005369676E6174757265206661696C6564B5
:1074A00020286572725F636F64653A2030782578B2
:1074B000290000005369676E61747572653A0000B7
:1074C000486173683A0000005075626C6963204B34
:1074D00065793A0068B60700496D61676520766591
:1074E00072696669656400002DE9F04104004FF09F
:1074F000010603D13349C420FBF748FF3248334A21
:1075000094F85410801AC008012202EB004541B1E2
:1075100094F8550040B1012806D0022804D0032871
:1075200002D028462AA147E01CB92649A320FBF730
:107530002DFF94F86E00032805D028462AA100F0FC
:1075400029FE14263BE094F8920018B194F89300B9
:10755000002834D1207A78B11C4A1B4B02209A1A99
:10756000D208E16800EB0247342908D0384623A14D
:1075700000F010FE112622E0284625A11CE020463E
:1075800003F0EAF830B1207880B12046FDF748F9E1
:1075900030B114E0384622A100F0FCFD12260EE0C6
:1075A000384623A100F0F6FD102608E094F85500B7
:1075B000012804D0284623A100F0ECFD0F26304618
:1075C000BDE8F08104C5070070CE070038CE070083
:1075D000496E76616C6964206669726D7761726567
:1075E00020747970652E0000496E76616C696420A4
:1075F0006861736820747970652E00004661756C4F
:1076000074792048572076657273696F6E2E00007A
:107610004E6F2048572076657273696F6E2E00009A
:10762000534420726571206E6F74206D65742E0056
:1076300046572076657273696F6E20746F6F206C89
:107640006F772E0046572076657273696F6E206DD6
:10765000697373696E672E000FB438B5040003D1E7
:1076600010A14220FBF792FE606918B90DA14320DA
:10767000FBF78CFE206818B90AA14420FBF786FEB0
:10768000606818B907A14520FBF780FE059900291D
:1076900005D006A800906A46204600F045F838BCA0
:1076A0005DF814FB2E2E5C2E2E5C2E2E5C2E2E5C96
:1076B0002E2E5C65787465726E616C5C66707269A2
:1076C0006E74665C6E72665F667072696E74662E4A
:1076D0006300000010B5040003D107A13120FBF7BF
:1076E00055FEA268002A05D0D4E904032168984712
:1076F0000020A06010BD00002E2E5C2E2E5C2E2ED1
:107700005C2E2E5C2E2E5C65787465726E616C5CEE
:10771000667072696E74665C6E72665F66707269BE
:107720006E74662E630000002DE9FC4791460C46FE
:107730005FEA000804D183A140F25220FBF726FE45
:10774000D8F8140020B97FA14FF41570FBF71EFE86
:10775000D8F8000020B97BA140F25520FBF716FEB7
:10776000D8F8040020B977A140F25620FBF70EFEAE
:10777000002C76D014F8011B39B125290ED04046D3
:10778000FCF7F2FC20780028F4D198F80C000028CF
:1077900067D04046BDE8FC47FFF79CBF00200122B0
:1077A00021782B291BD02D2902D0302908D102E0C5
:1077B00040F0010001E040F00200641C002AEFD11B
:1077C00000252A290ED02178A1F130020A2A11D2EF
:1077D00005EB850201EB4205641C303DF1E740F00A
:1077E0000400EAE7D9F800100B1DC9F80030096859
:1077F000641C0D44217800232E290BD114F8011F9D
:10780000A1F130020A2A05D203EB830201EB420305
:10781000303BF3E76C290DD068290BD0692921D0C2
:107820000BDC252918D0582931D063290ED06429C2
:1078300015D117E014F8011FECE7702969D07329FE
:1078400032D075291BD0782909D120E0D9F8000061
:10785000011DC9F8001001784046FCF785FC641C46
:1078600090E76CE0D9F800100A1DC9F800200968FB
:10787000CDE900500A224046FDF75CF9EFE7D9F860
:1078800000100A1DC9F8002009680A2206E0D9F88C
:1078900000100A1DC9F8002009681022CDE9005027
:1078A000404603F037FDDAE7D9F8001000270A1D3B
:1078B000C9F800200E68C00705D112E04046761CCA
:1078C0007F1CFCF751FC31780029F7D104E020211E
:1078D00040466D1EFCF748FCBD42C0D9002DF6D1D4
:1078E000BDE74EB13046F9F7BFFD074604E0202161
:1078F00040466D1EFCF738FCBD4206D9002DF6D17E
:1079000003E04046761CFCF72FFC31780029F8D1C3
:10791000A5E7D9F80000011DC9F80010056830215D
:107920004046FCF721FC78214046FCF71DFC08206E
:107930000021CDE90001034610222946B0E7BDE849
:10794000FC8700002E2E5C2E2E5C2E2E5C2E2E5CD4
:107950002E2E5C65787465726E616C5C66707269FF
:107960006E74665C6E72665F667072696E74665F76
:10797000666F726D61742E63000000002DE9F041A6
:107980001E4615460F46040003D11DA19E20FBF79D
:10799000FDFC206818B91AA19F20FBF7F7FC1DB960
:1079A00017A1A020FBF7F2FC39462046FBF7ECF9C3
:1079B00040B939462046FBF7E7F918B910A1A320D2
:1079C000FBF7E4FC60683946026820466A43FBF72F
:1079D000E4F958B960683946026820466A43FBF703
:1079E000DCF918B906A1A520FBF7D0FC20683346C6
:1079F0002A46D0F810C039462046BDE8F04160471D
:107A00002E2E5C2E2E5C2E2E5C2E2E5C2E2E5C637B
:107A10006F6D706F6E656E74735C6C6962726172AB
:107A20006965735C6673746F726167655C6E7266BC
:107A30005F6673746F726167652E630070B516467A
:107A40000C46050003D108A15520FBF79FFC1CB98B
:107A500005A15620FBF79AFC2C6031462846226887
:107A6000BDE87040104700002E2E5C2E2E5C2E2E9E
:107A70005C2E2E5C2E2E5C636F6D706F6E656E7467
:107A8000735C6C69627261726965735C6673746F52
:107A9000726167655C6E72665F6673746F72616750
:107AA000652E63002DE9F04128B1016819B1C9695B
:107AB000BDE8F04108470D4D0D480024461B142732
:107AC0000DE000BF04EB840005EB8000016829B1E4
:107AD000C969884710B10120BDE8F081641CB6FB7C
:107AE000F7F0A042EED80020F6E70000705A002020
:107AF000845A0020044801214174007A08B1002012
:107B00007047012070470000A87F0020012801D0A5
:107B1000032808D10449002201284A7400D000201B
:107B2000087402F00FBC7047A87F002070B50146B2
:107B3000022801D0032943D1224C207A00283FD0CB
:107B4000012831D002282FD11F48002302290068C4
:107B500002D0032928D119E0E360027912B1012A89
:107B600022D10BE0D0E90565721B142A00D3142240
:107B70002A4482614569AA420ED015E00169491C78
:107B80000161426991420FD1237213E0E268521CF5
:107B9000E260082A08D9E360237202290AD00D2185
:107BA000FCF7DDFD02F0C4FB607C28B1BDE870404D
:107BB00000F030BF0021F3E7BDE8704002F0C2BB27
:107BC00070BD0000A87F0020005A00202DE9F84376
:107BD0001D46089F16468846040003D12AA1882026
:107BE000FBF7D4FB1EB928A18920FBF7CFFB206847
:107BF00018B925A18A20FBF7C9FB1DB922A18B204A
:107C0000FBF7C4FB60684068B5FBF0F100FB115165
:107C100041B1B5FBF0F100FB115018B11AA18E2053
:107C2000FBF7B4FB4046FBF7A9F838B94046FBF731
:107C3000A5F818B914A19120FBF7A8FB3046FBF773
:107C40009DF838B93046FBF799F818B90EA1922083
:107C5000FBF79CFB2A4641462046FBF79EF848B9B5
:107C60002A4641462046FBF798F818B906A193200A
:107C7000FBF78CFB009720682B463246C7684146CD
:107C80002046B847BDE8F8832E2E5C2E2E5C2E2EA3
:107C90005C2E2E5C2E2E5C636F6D706F6E656E7445
:107CA000735C6C69627261726965735C6673746F30
:107CB000726167655C6E72665F6673746F7261672E
:107CC000652E630010B501684FF000004A0900D12D
:107CD000401E01F01F0201219140014204D104A184
:107CE0004FF4F670FBF752FB4FF0A04010BD0000C0
:107CF0002E2E5C2E2E5C2E2E5C2E2E5C2E2E5C6D7F
:107D00006F64756C65735C6E7266785C68616C5CE0
:107D10006E72665F6770696F2E68000030B5134B36
:107D2000014600201C6922460AE0D2681579854286
:107D300005D1401C0A28F6DB4FF0FF3030BD126839
:107D4000002AF2D1421CF9D0CA6810711A693AB1FE
:107D5000D268CC68126822601A69D268116030BD9E
:107D60001961C96800220A6030BD000054910020EA
:107D70007047FAF743BD704708B5034A00924023A5
:107D8000024A00F005F808BD3DA80700BC7F0020AE
:107D9000F0B595B01C4615460F4608461A9E00F0F1
:107DA0006BFB182109A8F9F754FB0E96CDE909548D
:107DB0000023082203A9384600F074FB05980690BA
:107DC000BDF81000ADF81C00BDF81200ADF81E00A3
:107DD00000208DF821000398082600F003000128F8
:107DE00002D0022818D032E003983346850AC0F347
:107DF000C2008DF8200003980FA9C0F38314A200DD
:107E0000384600F04FFB09A8009006AB22460FA9A8
:107E1000284600F08DFA1AE00398840DC0F3C200E2
:107E20008DF82000082C01D2254600E008253346B5
:107E30002A460FA9384600F035FB2E44641B09ABD7
:107E400006AA29460FA800F0D9F9002CEAD1384635
:107E500000F018FB15B0F0BD0A4A012902EBC00082
:107E600007D0022907D0032907D0042907D0002012
:107E700070470220704704207047007970474079AE
:107E80007047000038CE070010B5FFF772FF0421DD
:107E90000648FFF743FF002803DA05494120FBF7B6
:107EA00075FA02490120C968487110BD28CE070043
:107EB00090C907002DE9F04F8DB0FCF76DF918B1AE
:107EC00000200DB0BDE8F08F7D4E0020B061BFF303
:107ED0004F8FA6F580547B49A06801900D684FF044
:107EE0000009284004EB80000AE0B06970B96168BD
:107EF0000198814201D8A160E2E7284004EB8000AC
:107F00000C3001A9FCF769FE0028EED1002005AA7B
:107F1000A046019901EA050308EB8303491CDB68CD
:107F200042F82030401C01910228F2D3059800F05D
:107F30000300022802D001284CD0A8E00598502266
:107F4000810D8A46B2EB905F00D850210C4664F355
:107F50009F50059008315C4800F045FA070075D045
:107F600000F08AFA4B46082205A9384600F0C8FA04
:107F7000019909F1080B2940681A8000001D84420C
:107F800021D9524D30B1C2B208EB8101201A91467D
:107F90000C3104E02946E2B2002591462846C4B2DD
:107FA0005B46384600F0ACFA0BEB090325B12246DC
:107FB0002946384600F0A4FA01990AF1030001EBC2
:107FC000900001903BE008EB81015B462246384679
:107FD0000C31EFE70598C0F38310062800D3062084
:107FE000059960F38911C1F38310801C059181000C
:107FF000354800F0F8F9070049D000F03DFA4B464B
:10800000082205A9384600F07BFA09F10809002486
:108010000FE001984B4600EA0501401C08EB810186
:108020000190042238460C3100F06AFA09F1040983
:10803000641C0598C0F38310A042EAD837B13469B4
:10804000B06978B1384600F01DFA34E01FE0E0680E
:108050004079012804D122682046394612689047A9
:10806000E0680468002CF2D1384600F00BFA0020DA
:108070008DF800006846FBF7F9F8B06910B901996E
:10808000C8F808109DF80000FBF73CF913E03469CC
:1080900005E02168204689688847E0680468002C6C
:1080A000F7D10B480B49401AC008022101EB0040F0
:1080B00009A100F06FF8FCF76FF880F0010000E70D
:1080C00054910020145A0020BCCE0700608100208B
:1080D00088CE070038CE07004261636B656E64731B
:1080E00020666C7573686564000000002DE9F84F28
:1080F0008146264FD01C15468A46800800226946D4
:108100003E68FBF7D7FFDFF88880B0B3009CA01C67
:10811000009039683040091A8F003F1DBD4208EBBE
:10812000800002D82A46514608E03A4651460C30B3
:10813000F9F776F91648EA1B0AEB07010C30F9F754
:108140006FF94FEA1947FCF79BFA47EA0042601CB7
:10815000304008EB8000344008EB8401C260C868FE
:108160004FF6C07269F3C500904365F39F5020F04D
:108170000300801C20F00400C86098F8000001E0B3
:10818000FFF798FE0028FBD1BDE8F88F145A0020B5
:108190005481002000231A4602F0D4BE08B5012302
:1081A00000926A4602F0CEFE08BD1CB5CDE9002360
:1081B00002236A4602F0C6FE1CBD3EB5069C8DE851
:1081C0001C0003236A4602F0BDFE3EBD7FB5DDE91B
:1081D00008458DE83C0004236A4602F0B3FE7FBDEB
:1081E00070B586B00DF1280C9CE870008DE87C001D
:1081F00005236A4602F0A6FE06B070BD2DE9F047E1
:108200000E4680461C469246082940D894F80C90A9
:10821000002020731946104602F030F80025B542C0
:1082200006D218F805201BA12046FFF715FA03E037
:108230001AA12046FFF710FA6D1C082DEFD318A1E4
:108240002046FFF709FA0025B54212D218F805704A
:108250007E2F08D8F9F7E0F80068C05D10F03E0FF7
:1082600001D03A4600E02E220EA12046FFF7F4F995
:1082700003E00DA12046FFF7EFF96D1C082DE3D3B5
:1082800001222146504601F099FE84F80C90BDE889
:10829000F0870000202530327800000020202000E8
:1082A0007C0000002563000020000000064910B596
:1082B00000200870054800F0E3F8002803D10448C6
:1082C00000F0A2F9002010BD54810020BCCE0700B0
:1082D000A8BC070002480349401AC00870470000C4
:1082E000A8CE070038CE070013B56846FCF760FE3D
:1082F00008B100201CBD0248009950F831001CBD97
:1083000038CE070070B5094801250469A0F58050F2
:10831000057007E0E0684571216820464968884794
:10832000E0680468002CF5D170BD00005491002075
:108330002DE9FF4781460C9D00200C462F7B2873BA
:10834000984616462946184601F098FF072E42D255
:10835000DFE806F004090F161F2A360049462846B2
:10836000FFF77AF937E0494628462268FFF774F9A3
:1083700031E0D4E9002349462846FFF76DF92AE0A9
:10838000A0680090D4E9002349462846FFF764F925
:1083900021E0D4E90201CDE90001D4E900234946F6
:1083A0002846FFF759F916E004F1080007C88DE8E0
:1083B0000700D4E9002349462846FFF74DF90AE0B3
:1083C00004F108000FC88DE80F00D4E900234946E6
:1083D0002846FFF741F900222946404601F0EEFD0C
:1083E0002F73BDE8FF872DE9F041058A80462D1FD8
:1083F0004819C01CB0FBF5F0C6B24046FCF76AFE57
:10840000041E19D00020207101206071E580002732
:108410002546761EC4F800800BE04046FCF75AFE65
:1084200060B16179491C6171286005467F1CC0F804
:108430000080B742F1D32046BDE8F081204600F02D
:1084400002F80020F8E72DE9F041457901466B1E5E
:10845000002201E00968521C9A42FBD30F680146D2
:10846000002605E038460C68FCF79AFE2146761C8B
:10847000AE42F7D3BDE8F0810121001DFCF703BE39
:10848000FCF7D6BE10B504460121001DFCF71CFE0A
:1084900010F0FF0F04D12046BDE81040FFF7D3BF16
:1084A00010BD00001CB514460122CDE9002401AA2C
:1084B000FCF710FD0198A04204D003A14FF4807096
:1084C000FAF764FF1CBD00002E2E5C2E2E5C2E2EB3
:1084D0005C2E2E5C2E2E5C636F6D706F6E656E74FD
:1084E000735C6C69627261726965735C6D656D6FF6
:1084F000626A5C6E72665F6D656D6F626A2E6300A4
:108500001CB514460022CDE9002401AAFCF7E2FCC8
:108510000198A04203D002A1F620FAF737FF1CBD54
:108520002E2E5C2E2E5C2E2E5C2E2E5C2E2E5C6350
:108530006F6D706F6E656E74735C6C696272617280
:108540006965735C6D656D6F626A5C6E72665F6DA6
:10855000656D6F626A2E6300094902220A60BFF3EB
:108560006F8FBFF34F8F0A1D106006480268002A04
:10857000FCD000200860BFF36F8FBFF34F8F7047B0
:1085800004E5014000E40140094A01231360BFF300
:108590006F8FBFF34F8F0160064801680029FCD040
:1085A00000201060BFF36F8FBFF34F8F7047000044
:1085B00004E5014000E4014070B50E4C0123236046
:1085C000BFF36F8FBFF34F8F00230B4D08E000BF49
:1085D00051F8236040F823602E68002EFCD05B1C0D
:1085E0009342F5D300202060BFF36F8FBFF34F8F0E
:1085F00070BD000004E5014000E40140014800684E
:10860000C0B270471C0500408268002191608268FA
:108610001161826851618268D160826851608068AE
:108620000160704708B5002242504058009008BDD4
:1086300020B1034909680160002070470E2070478F
:108640002CBD07002DE9FE4307460E460846FFF7FE
:10865000EFFF00287CD100240094019406208DF8BF
:1086600000704FF00108ADF8040002948DF802800C
:1086700069462020326869DF3649374A891AC908B5
:10868000012202EB014530B100F09EFA0246284675
:108690003249FFF783FD00948DF801808DF8024088
:1086A000019402948DF8034069464020326869DFE6
:1086B00030B100F089FA024628462949FFF76EFDDD
:1086C00000948DF80070F720ADF802000194029438
:1086D00069462320326869DF30B100F075FA02463E
:1086E00028462049FFF75AFD0094019402948DF822
:1086F000008069460120326869DF30B100F064FA19
:10870000024628461849FFF749FD4FF4B060009033
:10871000019402946946A120326869DF30B100F00B
:1087200053FA024628461149FFF738FD0094019498
:1087300002948DF800406946A020326869DF30B1AC
:1087400000F042FA024628460949FFF727FD0020BB
:10875000BDE8FE8398CE070038CE070088CB07001F
:10876000D0CB07001CCC0700E8CA070034CB0700B9
:1087700094CA07002DE9F0410546076860DF80468E
:1087800019491A482A68081AC608BA4219D9022093
:1087900000EB064416A12046FFF7FCFC20463A46B3
:1087A0001FA12B68FFF701FD4FF08050D0F80C019E
:1087B0002968800200F10050421A204625A1FFF7E7
:1087C000EDFCB8F100004FF001040AD000F0FCF914
:1087D000024604EB06402AA1FFF7E0FC4046BDE854
:1087E000F0812F480470F9E798CE070038CE0700D3
:1087F000496E73756666696369656E742052414D92
:1088000020616C6C6F636174656420666F722074A4
:10881000686520536F66744465766963652E000051
:108820004368616E6765207468652052414D20730E
:1088300074617274206C6F636174696F6E2066720C
:108840006F6D203078257820746F20307825782E51
:10885000000000004D6178696D756D2052414D201A
:1088600073697A6520666F72206170706C696361EC
:1088700074696F6E20697320307825782E000000AF
:1088800073645F626C655F656E61626C6528292048
:1088900072657475726E65642025732E0000000089
:1088A0006B5A002030B51848ADF5017D00780028DE
:1088B00026D04FF4FA7400BFADF8004280A9684694
:1088C00061DF38B105281BD00DF5017DBDE83040D2
:1088D000FAF78ABB6D460D497DA800F0F1F809E072
:1088E0007DA800F0D5F8D0E90021284690477DA862
:1088F00000F024F97DA800F0CBF80028DCD0EFE7E9
:108900000DF5017D30BD00006B5A002030BD070021
:10891000F8B5134C2078C0B10120A07001F058FFC9
:10892000112814D0022001F06FFF00258DF80050AF
:108930006846FAF79BFC11DF064625709DF800009B
:10894000FAF7E0FC2EB13046F8BD0820F8BD002053
:10895000F8BDA57002F016FA032001F055FFF6E706
:10896000685A00207CB5194C207808B108207CBDDD
:108970000120A070002001F02BFF112819D0002049
:1089800001F042FF12480026006801908DF8006057
:108990006846FAF76BFC0F4901A810DF05000AD002
:1089A000002020709DF80000FAF7ACFC2DB128469D
:1089B0007CBD00207CBD0120F3E7A670667002F04C
:1089C00045FA012001F020FFF3E70000685A00207B
:1089D000C4BC0700852F07000EB50A49684600F0A1
:1089E0006FF808E0684600F047F8D0E900108847C3
:1089F000684600F0A3F8684600F03EF80028F1D180
:108A00000EBD0000E0BC0700014800787047000080
:108A1000685A00200548817819B1007818B1FFF72D
:108A200077BF08207047FFF79DBF0000685A0020FD
:108A30001FB568464BDF30B1052819D004B0BDE83A
:108A40001040FAF7D1BA0B4901A800F039F809E053
:108A500001A800F029F8D0E900210098904701A86A
:108A600000F06CF801A800F01FF80028E1D0EFE753
:108A70001FBD00004CBD070010B5040003D1034921
:108A8000C420FAF783FCA06810BD000040CA0700AC
:108A900010B5040003D10349C420FAF777FCA0689D
:108AA00010BD000040CA070010B5040003D10349FF
:108AB000C420FAF76BFCA06810BD000040CA070094
:108AC00070B50D46040003D108495020FAF75EFC4A
:108AD0001DB906495120FAF759FC256028686060E5
:108AE0002046BDE8704000F003B8000050C5070004
:108AF00010B5040003D110493320FAF747FC206871
:108B000018B90D493420FAF741FC606818B90A49D0
:108B10003520FAF73BFCD4E900104A68904201D1B5
:108B2000002004E0D0E900239A4202D01046A06061
:108B300010BD08306060F0E750C5070010B50400B4
:108B400003D112496320FAF721FC206818B90F49B4
:108B50006420FAF71BFCA068002815D021688968FA
:108B60000844A060606818B908497320FAF70EFC41
:108B7000D4E901014268914206D108306060204684
:108B8000BDE81040FFF7B4BF10BD000050C507009E
:108B90000C4A10B502F594730EE0991AC91001EB56
:108BA000D171491002EBC1010C68844201D90B4616
:108BB00002E005D201F108029A42EED3002010BD76
:108BC000486810BD68BA070000B5FFF7E1FF00284C
:108BD00000D1014800BD000054BA07002DE9F04162
:108BE00004461348134BC01A0C21B0FBF1F6A069E0
:108BF0004FF0FF3110F8022C02B92169002011E07A
:108C000000EB400503EB85052F68974209D14F1C07
:108C100002D06F688F4204D194E80F00AD68A84776
:108C200003E0401CB042EBD301202060BDE8F0819E
:108C30000CCF070000CF070010B5144612680830AB
:108C4000202A02D248F2145010BD002201F028FF61
:108C50000028F9D120202060002010BD083001F04C
:108C6000A7BF083002F064B802480068002800D0AE
:108C7000012070470004014070B50C46050004D186
:108C80000F494FF48270FAF781FB24B90C4940F286
:108C90000510FAF77BFB0B480B49401AC00804216A
:108CA00001EB004009A1FFF775FA13490320C968D9
:108CB00088476869FEF726FAFBF77BFD607070BD98
:108CC000DCC0070050CE070038CE070048616E6454
:108CD0006C65204E52465F4446555F4F505F4F4291
:108CE0004A4543545F4352454154452028636F6DC4
:108CF0006D616E6429000000C859002070B50D46F2
:108D000020B916494FF49670FAF740FB25B913497C
:108D100040F22D10FAF73AFB11481249401AC108E7
:108D2000042000EB014004460FA1FFF733FA194974
:108D3000081FFEF701FAFBF73CFD6870012805D11A
:108D40000020FDF7A9FF10B10A20687070BD204611
:108D5000BDE8704010A1FFF71DBA0000DCC007009D
:108D600050CE070038CE070048616E646C65204E17
:108D700052465F4446555F4F505F4F424A45435409
:108D80005F455845435554452028636F6D6D616EAE
:108D900064290000D059002057726974696E6720F9
:108DA00076616C696420696E697420636F6D6D61B2
:108DB0006E6420746F20666C6173682E0000000082
:108DC00070B50D46040004D11A494FF48970FAF7C2
:108DD000DDFA206920B9174940F21310FAF7D6FAE4
:108DE000A08A20B913494FF48A70FAF7CFFA25B94F
:108DF000104940F21510FAF7C9FA0F480F49401A06
:108E0000C008042101EB00400DA1FFF7C3F9A18ABE
:108E10002069FEF733F9FBF7CCFC68702846FBF7B6
:108E2000C7F9E168002903D02069BDE87040084710
:108E300070BD0000DCC0070050CE070038CE070030
:108E400048616E646C65204E52465F4446555F4FE4
:108E5000505F4F424A4543545F575249544520287A
:108E6000636F6D6D616E64290000000030B587B0DE
:108E70000C46054618221B496846F8F7D1FA207BB4
:108E80000195194D8DF80000012806D0022815D053
:108E9000062821D1607B04901EE0A888E880607BD2
:108EA0000490617CD4F80E0061F31F600590049873
:108EB000012811D10D48FDF703FF0DE00C480D49C5
:108EC000401AC008042101EB00400BA1FFF762F932
:108ED000B4F80D00A880E8806846FDF7E7FB07B00E
:108EE00030BD0000F8B80700A859002020CE0700C8
:108EF00040CE070038CE0700536574207265636565
:108F0000697074206E6F74696600000070B50E465B
:108F10000B480C49401AC108042000EB01440AA187
:108F20002046FFF737F9114D204611A1AB6C2A6D91
:108F3000FFF73BF9A86CB060286D706070BD000051
:108F400050CE070038CE070048616E646C65204E35
:108F500052465F4446555F4F505F4352435F47451B
:108F60005420286461746129000000003C760020D0
:108F70004F66667365743A25642C204352433A3039
:108F800078253038780000002DE9F84F0D46074667
:108F9000374838494FF00409401AC40809EB044027
:108FA000064635A1FFF7F6F8FEF738F9012101EB87
:108FB00004444FF0080AA8B17A694FF00308B2B12F
:108FC00037493848130515D0436DD1F808C013440C
:108FD00063450FD0204634A1FFF7DCF885F8018007
:108FE000BDE8F88F204639A1FFF7D4F819E02046F4
:108FF00044A1F1E7B2F5805F06D9204648A1FFF70A
:10900000C9F885F80190EBE7436DD1F808C003EB90
:109010000208E04508D920464A49CDF800C0FFF7CC
:10902000CCF885F801A0DBE74264C26C03650363FA
:10903000804682647869002200F6FF70070B48685A
:1090400039461844FDF740F930B120463EA1FFF7FC
:10905000A1F805206870C3E7D8F8481000913046A1
:109060003FA1D8F85030D8F84420FFF7A6F8B7E76A
:1090700050CE070038CE070048616E646C65204E04
:1090800052465F4446555F4F505F4F424A454354F6
:109090005F435245415445202864617461290000B2
:1090A000C85900203C7600204F626A6563742073C3
:1090B000697A65206D7573742062652070616765DB
:1090C00020616C69676E65640000000043616E6E2C
:1090D0006F74206372656174652064617461206FD0
:1090E000626A65637420776974686F75742076614D
:1090F0006C696420696E697420636F6D6D616E6464
:10910000000000004F626A6563742073697A65200D
:1091100063616E6E6F7420626520302E0000000067
:10912000496E76616C69642073697A6520666F7236
:10913000206F626A6563742028746F6F206C61729F
:109140006765290068C007004572617365206F700C
:1091500065726174696F6E206661696C6564000098
:109160004372656174696E67206F626A656374201B
:10917000776974682073697A653A2025642E204FD8
:1091800066667365743A203078253038782C204331
:1091900052433A2030782530387800002DE9F041EC
:1091A0000E46074615481649401AC508042000EB2C
:1091B000054014A1FEF7EEFF1C4CD4E91401626CCB
:1091C000431A9A420AD0012000EB054018A1FEF78D
:1091D000ECFF082070700120BDE8F081002161647F
:1091E000A16CE16460650021384600F035F819494A
:1091F0000420C96888470020EEE7000050CE070031
:1092000038CE070048616E646C65204E52465F445C
:1092100046555F4F505F4F424A4543545F4558455E
:109220004355544520286461746129003C76002030
:10923000496E76616C696420646174612E20657882
:109240007065637465643A2025642C20676F743AF6
:1092500020256400C8590020F0B5044687B00020DE
:10926000FEF720FC01002548254A4FF00107A0EB3E
:1092700002004FEAD0050AD0224A18212046F9F709
:109280006FFF020037D007EB05401FA131E0182225
:1092900028496846F8F7C4F82748284E184B174D58
:1092A000016DEB1A0420DB08B26800EB0345914224
:1092B00015D1284622A1FEF76DFFD6E90101FDF781
:1092C000B9FD8DF80100FBF774FA8DF80100D4E9BF
:1092D0000112684690472648FDF7DEFC05E08DF850
:1092E0000170D4E90112684690479DF80120284694
:1092F00020A1FEF753FF07B0F0BD000050CE0700DD
:1093000038CE0700599207004661696C6564207485
:109310006F207363686564756C65206F626A65634E
:109320007420657865637574653A20307825782EE9
:1093300000000000B8B907003C760020C8590020A2
:1093400057686F6C65206669726D77617265206918
:109350006D6167652072656365697665642E20506E
:109360006F737476616C69646174696E672E000056
:109370002D950700526571756573742068616E6480
:109380006C696E6720636F6D706C6574652E20521A
:109390006573756C743A20307825780038B50D46C1
:1093A0000C480D49401AC108042000EB0140044656
:1093B0000AA1FEF7EFFE134813A1826CAA60036DA9
:1093C0004FF480506B60E86000902046FEF7F5FE99
:1093D00038BD000050CE070038CE070048616E64EB
:1093E0006C65204E52465F4446555F4F505F4F427A
:1093F0004A4543545F53454C4543542028646174A7
:10940000612900003C760020637263203D203078A3
:1094100025782C206F6666736574203D2030782592
:10942000782C206D61785F73697A65203D203078F3
:10943000257800002DE9F0410E46044626482749CC
:10944000401AC708042000EB074025A1FEF7A2FE42
:10945000FDF7E4FE90B12C4DD5E91401401AA18A24
:109460006A6C084490420BD9012000EB074027A109
:10947000FEF790FE03207070BDE8F0810820FAE747
:10948000284A286B526800EB02081F4A20694832BC
:10949000FAF7A0FE0746E06820B923494FF4F870B8
:1094A000F9F774FFD4E90331A28A4046FCF7C2FF02
:1094B00020B1D4E90310BDE8F0410847A18A286B28
:1094C00008442863A18A286DAF6408442865B76002
:1094D000286D7060D0E7000050CE070038CE07003E
:1094E00048616E646C65204E52465F4446555F4F3E
:1094F000505F4F424A4543545F57524954452028D4
:1095000064617461290000003C7600205772697420
:1095100065207265717565737420746F6F206C6F50
:109520006E670000C8590020DCC0070008480949E0
:1095300010B5401AC008042101EB004006A1FEF757
:1095400029FE12490620C968BDE8104008470000FE
:1095500050CE070038CE0700416C6C20666C6173FA
:1095600068206F7065726174696F6E7320686176D0
:109570006520636F6D706C657465642E204446557C
:1095800020636F6D706C657465642E00C85900208F
:10959000FEF7B8FEFEF78EFC0028FBD10D4E6425C9
:1095A0004FF47A47741C3846A0476D1EFAD10A481A
:1095B0000068C00700D000BEBFF34F8F0648E438F4
:1095C0000168064A01F4E06111430160BFF34F8F67
:1095D00000BFFDE760B60700F0ED00E00400FA050B
:1095E00010B50446084809492246401AC00804211B
:1095F00001EB004006A1FEF7D1FD2146BDE8104079
:109600000848FBF7CDBD000040CE070038CE07006C
:1096100046726565696E67206275666665722025AB
:1096200070000000A8CE070030B58A1D8B79083184
:1096300087B0022B33D153888489A3422FD1127A69
:10964000012A2CD1184C0DF1040C3CCC8CE83C00C8
:109650000A89ADF80C204A890C3104911249ADF801
:109660000E208039114C096A0591CDF818D0018A75
:1096700005AA6088ADDF18B96846FAF7E1FB38B192
:109680000020ADF8080001A96088B0DF50B106E005
:1096900040F2FD10ADF8080001A96088B0DF00209D
:1096A00007B030BD0120FBE710B90700A859002022
:1096B00070B506468C1DC888B18888B088422DD107
:1096C0001B48FBF707FD05001A481B49A0EB0100EA
:1096D0004FEAD00024D0F4210091042101EB004096
:1096E00063892A4615A1FEF768FD628904F10C0121
:1096F0002846F7F795FE1822184901A8F7F790FEBB
:10970000029605956089ADF8180001A8FCF7CEFF18
:10971000002803D029460648FBF742FD08B070BD7B
:10972000022101EB00400EA1FEF734FDF6E7000038
:10973000A8CE070040CE070038CE07004275666607
:1097400065722025702061637175697265642C20D3
:109750006C656E20256420282564290020B9070047
:1097600063616E6E6F7420616C6C6F6361746520F1
:109770006D656D6F72792062756666657221000095
:10978000F8B50D4614460646694600F057FA00281B
:109790000FD0009BB3F5803F0AD2981C834207D8B4
:1097A000A9780222B2EB911F02D02989814201D20D
:1097B0000020F8BD2380A11C3046009A00F094FBE5
:1097C000F8BD114600F0D6B8114600F0E3B8F8B580
:1097D0000C4615460646694600F030FA00280CD0C3
:1097E000009A501C904207D3A1780223B3EB911F3B
:1097F00002D02189814201D20020F8BD294630469D
:1098000000F072FB009A0021A954F8BD2DE9FF4138
:109810000C46CE6817460546694600F037FB00281F
:109820000ED0E06800280BD0A0783A46C0F30110B3
:1098300002283146684606D000F0DAF801996960DE
:1098400004B0BDE8F08100F086F8F7E77CB50D467E
:109850001446694600F08FF9002820D0288908288E
:1098600006D0042809D002280AD001280CD015E01F
:10987000DDE90001C4E900010AE00098206006E08B
:10988000009800B2208002E0009840B22070C1171A
:10989000DDE9002350405940084301D000207CBD41
:1098A00001207CBD7CB50D461446694600F0A1F947
:1098B000002820D02889082807D00021042809D0B2
:1098C00002280AD001280CD014E0DDE90001C4E927
:1098D000000109E00098206006E0009880B2208036
:1098E00002E00098C0B22070DDE9002350405940EA
:1098F000084301D000207CBD01207CBD7CB50D4615
:109900001446694600F075F9002821D029890829F4
:1099100008D00098C21704290BD002290DD00129C4
:109920000ED014E0DDE90002C4E90002014613464E
:1099300009E0C3170146206005E001B2218001E083
:1099400041B22170CB1741405340194301D0002050
:109950007CBD01207CBD70B50D46064614461146FF
:10996000284600F0AEFA224629463046BDE870404F
:1099700000F03EB838B50C460422694600F0B4FA4F
:10998000002806D09DF80310009861F31F60206046
:10999000012038BD1CB50C460822694600F0A4FA27
:1099A000002824D09DF801109DF800209DF8023079
:1099B000080E42EA012242EA034240EA13409DF8BF
:1099C00003309DF8041040EA132008439DF8051069
:1099D00042EA036240EA01209DF8061040EA014095
:1099E0009DF8071040EA0160C4E9002001201CBD79
:1099F0002DE9F04F04469DB00020009006460190EE
:109A00004FF0FF3A0AA800F07DF94FF0010BE9464C
:109A100082E012AB05AA06A9204600F0C9F850B1B1
:109A20000AA8059900F07FF960B10B98807810F0D2
:109A3000300F53D060E09DF84800002870D11DB071
:109A4000BDE8F08F0598B04242D30B9D0AAE0B984B
:109A5000807800F00F00082812D0304600F07AF924
:109A60000B98A842F3D156460599B14230D3D4F8A9
:109A7000088009919DF8181008910E990D6820E052
:109A80000B980688F0E729680F682FB1DDE90832E6
:109A900029462046B84711E011948968DDE908722B
:109AA000098891420CD1294617A8FBF72BF985F8B4
:109AB0000CB017AA39461198FAF725FC0028BED039
:109AC000AD6815B1A1684145DDD0A168414523D1FC
:109AD0009DF81810204600F043FA1BE00C9840282F
:109AE0000AD200F01F010BFA01F00C994A0959F84B
:109AF0002230034349F82230E5682DB10AAB9DF8C6
:109B0000182020460599A8470AAA9DF81810204653
:109B1000FAF7F9FB002892D0A06800287FF479AF0B
:109B2000DDE90B0485780AA800F014F90028F7D1C4
:109B300015F0300F03D10B98008800B1641CC4B13C
:109B40000020494605E000BF51F82020521C0ED1EC
:109B5000401CB0EB541FF7D3600959F8201004F0F3
:109B60001F00C0F120022AFA02F0814201D0002039
:109B700065E7012063E71CB50C46694600F039F83B
:109B8000002814D0DDE90002C10709D051084FEACE
:109B900030006FEA00026FEA0100C4E9002004E02F
:109BA00051084FEA3000C4E900014FF001001CBD2C
:109BB000F8B507460020187008700E4610601C4665
:109BC00015466946384600F039F801004FF00100AB
:109BD00009D0009959B1C8082860009800F0070022
:109BE00030700120F8BDB96809B10020F8BD2070BF
:109BF000FBE72DE9F8430026884681463446354682
:109C000004E0402E02D30020BDE8F88369464846B0
:109C100000F096F90028F7D09DF80070324607F062
:109C20007F00C10FF7F7E8FB29430443F61D0D46FB
:109C30003806E6D4C8E900410120E5E7F8B50E464C
:109C40000746694600F07CF900280AD09DF80040DC
:109C5000200616D5072504F07F0403E0202D01D34C
:109C60000020F8BD6946384600F06AF90028F8D0AF
:109C70009DF8001001F07F00A8400443ED1D080688
:109C8000ECD401203460F8BD30B45968114AC96879
:109C9000914208D1D0E901120F48D0E901342343A1
:109CA00003D00021817030BC704711F8013BA2F154
:109CB00001021B06F9D4C0E9011201218170074895
:109CC000074930BC401AC008042101EB004005A13F
:109CD000FEF764BA40B70700DC59002068CE0700E1
:109CE00038CE070050423A20496E69742070616393
:109CF0006B65742064617461206C656E3A20256424
:109D000000000000C26000230160C0E901138B88DD
:109D10001A440261B1F906301A44426108880028E9
:109D200000D00120704770B545680E460446606853
:109D30000188B14206D1807800F00F00082801D0D8
:109D4000012070BD204600F005F86068A842EED101
:109D5000002070BD30B541680A885AB101F1100386
:109D600043600A8A42B18C780A89C4F30115032D35
:109D700007D00BE0002030BDC2680168FFF7C2FFCA
:109D8000F8E79D78C5F30115032D06D00225B5EB44
:109D9000141F08D14C89624309E08D8804690022B0
:109DA000641B046103E0B5EB941F00D104228978A1
:109DB00011F0300F02D18168491C81609C880169D3
:109DC000214411440161B3F906201144416101208D
:109DD00030BD30B54168002487B0897801F00F02AA
:109DE000082A11D08A091ED00222B2EB911F09D194
:109DF0000269C1F301110229146001D0032901D1C4
:109E00004069048007B030BD0069056808E02C7324
:109E100029466846FAF776FF6846FFF7DAFFAD682D
:109E2000002DF4D1EEE7C1F30111012912D002296E
:109E3000E6D00329E4D04268917801F00F010729A8
:109E40000BD0D16881B11289006907B0BDE83040FC
:109E5000F7F7E6BA41690C70EDE70169D06807B021
:109E6000BDE8304000F02DB81189006907B0BDE8A9
:109E70003040F7F7EEBA000010B5034B002408C0DD
:109E800080E8160010BD00004D41070038B50D46B2
:109E900004466946FFF7D2FE00280BD0D4E9000241
:109EA000D4E90213C5E90002C5E902130098814212
:109EB00001D2002038BDA860A168081AA060012066
:109EC00038BD00B50A4687B001466846FFF71AFF5D
:109ED000002807D06846FFF77CFF6846FFF73AFF87
:109EE0000028F7D107B000BD7FB514460546A9B9D3
:109EF000124A2868904208D110E01022694628468C
:109F0000FFF7F2FF002807D0103C102CF5D82246AE
:109F100069462846FFF7E8FF04B070BDA868A04274
:109F200001D20020F8E72B682246284698470028EF
:109F3000F2D0A868001BA8600120EDE74D410700A2
:109F400010B504468068002809D023680122204605
:109F50009847002803D0A068401EA060012010BDD3
:109F600038B5002439B1012912D0022912D00529AF
:109F70001DD0002038BD0546012269462846FFF75E
:109F8000B3FF90B19DF800000006F5D4012038BD64
:109F900008220DE005466946FFF750FE28B1002172
:109FA0002846009AFFF7A0FF38BD204638BD04229E
:109FB000BDE838400021FFF797BF000010B50C4600
:109FC000017A052908D0407A38B1084808A102680A
:109FD0002046FDF741FB00E01AB106A12046FDF73F
:109FE0003BFB2046BDE81040FDF774BB445A0020FF
:109FF000257300000D0A00002DE9FC41804622482F
:10A0000017460E46C5680A46012441462846FAF717
:10A01000F1FB70B195F8550068B100F00101C0F393
:10A02000400243462846CDE9006700F089F848B170
:10A0300009E0172407E03B4632464146284600F037
:10A0400027F8F4E70524114D6FB1012C13D005F169
:10A050002400FBF7D3FE00BFFCF722FDC5F84880C3
:10A060002046BDE8FC81012C02D0FCF719FDF7E782
:10A0700001206861F4E7002231464046FAF7AAF869
:10A08000C5E90960E8E70000DC5900203C760020C3
:10A090002DE9F041044690F8550094B01D4617464E
:10A0A000884620B1174940F22730F9F76FF90126A9
:10A0B000CDE9007643460022214602A8F9F742FF87
:10A0C00000281CD0D5B1412202A90F48F7F7A8F902
:10A0D0000F4810490D4D401AC008042101EB004003
:10A0E0000DA1EE62FEF756F80020286294F8920067
:10A0F00010B194F8930008B96068A860012014B00A
:10A10000BDE8F081BCC40700DD7800203C7600206B
:10A1100068CE070038CE0700496E76616C696461CD
:10A1200074696E67206F6C64206170706C69636124
:10A1300074696F6E20696E2062616E6B20302E0034
:10A140002DE9FF4FA5B0884604461546442113A8C3
:10A15000329FF7F77EF9442102A8F7F77AF9DDF884
:10A16000A09058EA050004D13C4940F26130F9F76B
:10A170000DF93B483B4A801A02224FEAD00A02EB13
:10A180000A46B8F1000F1ED0A16D289800F01AFE03
:10A19000002848D02898FAF74BFD4FF0010B20B16A
:10A1A00030463149FDF7F6FFB5B3A16DCDE9001B8F
:10A1B0000022214613A8289BF9F7C4FE002832D0BC
:10A1C000A06D81443F1A8DB10020CDE900704B464F
:10A1D0004246214602A8F9F7B5FE002823D09DF893
:10A1E000080018B130462149FDF7D4FF339898B3E1
:10A1F0001F4EB8F1000F1ED02898FAF719FD18B1BC
:10A2000006F11800FBF7FAFD412213A91948F7F7E8
:10A2100007F95DB1AC200AE0FFE70BEB0A401649F5
:10A22000FDF7B8FF002029B0BDE8F08FA520F0624F
:10A23000A06D706301E0AA20F0626DB10D4841226B
:10A2400002A98230F7F7ECF894F8920010B194F874
:10A25000930008B96068F0600120E4E7BCC407001F
:10A2600068CE070038CE070078C4070074C3070023
:10A270003C7600209C780020C0C2070038B5C38817
:10A280000D46044633B114A0009015A216A128462D
:10A29000FDF7E2F9217A05291CD0607A48B1A0883F
:10A2A000FDF7DAFD164951F8202016A12846FDF7E2
:10A2B000D3F9A0880021FEF717F803461049207A49
:10A2C000143951F8202001B02846BDE830400EA1D5
:10A2D000FDF7C2B938BD00001B5B306D0000000007
:10A2E0001B5B313B33316D0025734C6F677320640A
:10A2F000726F70706564202825642925730D0A002B
:10A30000445A0020257300003C25733E2025733AF3
:10A3100020000000EFF30580C005C00D01D0012032
:10A320007047EFF3148040F30000401C70470000BA
:10A33000034802490068FAF779BE0000045A002079
:10A3400024BA07002DE9F041224C0025224E207A44
:10A35000012730B92148311D0068FAF772FE3060DC
:10A3600038B1022020723168087928B101281BD148
:10A3700013E06560BDE8F081D1E90503C01A142837
:10A3800000D31420820806D082080869C9681844DE
:10A39000194429DF05E00122F7E7D1E90301084468
:10A3A00028DF58B1112812D003213068FAF7D7F905
:10A3B00025726560BDE8F041FFF7BABF207C002838
:10A3C000D8D1BDE8F04100210220FDF7AFBB2772D4
:10A3D000D0E70000A87F0020005A002024BA070020
:10A3E00010B5074C201DFAF74BFE002806D1607C03
:10A3F000002803D1BDE81040FFF7A4BF10BD000046
:10A40000A87F002010B510461A46F7F709F800207B
:10A4100010BD10B510461A46F7F702F8002010BD1F
:10A420002DE9F0411E681C461546074621B1012959
:10A4300018D0052923D119E000202060401C20609D
:10A44000B0421CD8012229463846FFF74DFD0028AE
:10A4500006D015F8010B000601D52068EEE70120B3
:10A46000BDE8F08108200246186002E004200246A0
:10A47000186029463846BDE8F041FFF735BD002099
:10A48000EEE770B516460A460446C11C104600F0B9
:10A490001FFF054661193046C91C00F019FF28440A
:10A4A00070BD000003B5094A85B0D2E91612CDE9A6
:10A4B000001207498989ADF8001006A9CDE90210FC
:10A4C000044869464088AEDF07B000BD90B8070079
:10A4D000E05E0020A85900200846704708467047F3
:10A4E0002DE9F047FCF7E8FBDFF8C480D8F830200E
:10A4F000D8F8347000EB020AB81A411EC1F30B0100
:10A50000401A00F6FF792B492B48D8F84860081A02
:10A51000C508042000EB0540044628A1FDF73AFEDB
:10A5200042F204002F4A8159012000EB0545914277
:10A5300006D028462CA1FDF72DFE0320BDE8F087AC
:10A54000D8F830000644B84205D1204633A1FDF7C3
:10A5500021FE0020F2E7C0B906F500500178142969
:10A5600001D9416900E000213148B1FBF0F34FF41B
:10A5700040510A78142A01D9496900E00021B1FB51
:10A58000F0F220462BA1FDF710FE08234A46314683
:10A590005046FAF7D5F9040005D0284630A1FDF75A
:10A5A000F9FD2046CAE7BDE8F0470020FCF774BB80
:10A5B0003C76002088CE070038CE0700456E7465D3
:10A5C00072206E72665F626F6F746C6F6164657229
:10A5D0005F6466755F73645F636F6E74696E7565E3
:10A5E00000000000DBE5B151536F757263652061B7
:10A5F00064647265737320646F6573206E6F74207A
:10A60000636F6E7461696E20612076616C6964208D
:10A61000536F66744465766963652E005344206108
:10A620006C726561647920636F7069656400000015
:10A6300040420F005570646174696E672053442E68
:10A64000204F6C64205344207665723A2025642C98
:10A65000204E6577207665723A2025640000000060
:10A660004661696C656420746F20636F7079206641
:10A6700069726D776172652E0000000070B50F4839
:10A680000F49401AC408042000EB04400DA1FDF757
:10A6900081FDFFF725FF05004FF0010000EB0444AA
:10A6A00002D020460FA105E0F8F77AFE050004D09D
:10A6B000204612A1FDF76EFD284670BD88CE07002A
:10A6C00038CE0700456E746572206E72665F6466F0
:10A6D000755F73645F626C5F636F6E74696E7565DE
:10A6E0000000000053442B424C3A20534420636F37
:10A6F0007079206661696C656400000053442B42E8
:10A700004C3A20424C20636F7079206661696C6519
:10A7100064000000F0B50546002003464FF44054A5
:10A720000C4E4FF6FE7712E0D4F804C0B44505D1C4
:10A7300055F823C0B4F80CE0F44504D02AB155F81C
:10A7400023C0BC4501D10120F0BD5B1CDBB28B42B4
:10A75000EAD3F0BDDBE5B15110B5040003D11A49CD
:10A760005320F8F713FE4FF44050184940688842D0
:10A7700021D1218A71B1626904F11400002A94F890
:10A7800055200BD0042A07D00022BDE81040C9B2E2
:10A79000FFF7C0BF002010BD0122F6E712B1012A69
:10A7A00007D1F7E7012904D9C9B20022FFF7B2FFA8
:10A7B000F0E7012010BD208A10B160690028E9D1BE
:10A7C00020780028F5D110BD04C50700DBE5B151A4
:10A7D0003EB504460B496846FEF772F90AE0684642
:10A7E000FEF74AF9D0E900212046904740B168467B
:10A7F000FEF7A4F96846FEF73FF90028EFD13EBD09
:10A8000011203EBDC8BC07003EB504460A49684653
:10A81000FEF756F909E06846FEF72EF9D0E9002167
:10A82000204690476846FEF789F96846FEF724F906
:10A830000028F0D13EBD0000D4BC07002DE9F04156
:10A840001400884618D000250E4F032608EB05019A
:10A8500022460020F7F7D4FF0544241A40B938787F
:10A86000002809D008494FF47A408847761E05D061
:10A8700001203870002CE9D1BDE8F081002038704B
:10A88000FAE70000085A0020A1BC07002DE9F041BA
:10A890000E46074613481449144D401AC4080320B5
:10A8A00000EB044012A12A68FDF778FC3046F9F766
:10A8B000AFFC20B919494FF4C170F8F767FD184B88
:10A8C0003A463146286800F053F8020007D00120CC
:10A8D00000EB0440BDE8F04112A1FDF75FBCBDE80C
:10A8E000F081000058CE070038CE0700D85900206C
:10A8F0004261636B696E672075702073657474695B
:10A900006E6773207061676520746F206164647284
:10A9100065737320307825782E00000034C207005C
:10A92000BC720020436F756C64206E6F742070657C
:10A9300072666F726D206261636B7570206F662046
:10A94000626F6F746C6F6164657220736574746993
:10A950006E677321204572726F723A2030782578C5
:10A960000000000000225821001DF9F733BC000050
:10A970002DE9F04715464FF460771E46894680461C
:10A980003A46F6F778FD224A224B0421D21AD20821
:10A9900001EB02440028204617D01FA1FDF7FAFB67
:10A9A0002046424621A1FDF7F9FB00220121404645
:10A9B000FBF78AFC174A164B01219A1AD20801EBC1
:10A9C000024458B1204621A11DE02949FDF7E2FBD0
:10A9D0000DB10020A8470020BDE8F08726B9254921
:10A9E00040F25D10F8F7D2FC3A4649463046F6F799
:10A9F00017FD2B463A4631464046FBF71BFD002823
:10AA0000EAD020461CA1FDF7C5FB0320E4E70000C7
:10AA100058CE070038CE070057726974696E6720F8
:10AA200073657474696E67732E2E2E0045726173A0
:10AA3000696E67206F6C642073657474696E6773E8
:10AA40002061743A2030782530387800436F756C77
:10AA500064206E6F74206572617365207468652070
:10AA600073657474696E6773207061676521000097
:10AA7000E8C1070034C20700436F756C64206E6F35
:10AA80007420777269746520746865204446552087
:10AA900073657474696E6773207061676521000067
:10AAA00070B516460D46040007D035B1206C8022E3
:10AAB00000213828225403D307E00E2070BD215412
:10AAC000401C3828FBD30BE02154401C4028FBD30A
:10AAD0002146084600F096F838212046F6F7B9FCE2
:10AAE000216CD4E912304A0FC9003834591850414A
:10AAF000C4E90410227CE2710A0A42EA0062A271EF
:10AB00000A0C42EA00426271020242EA11602071BC
:10AB10006069E070010AA170010C6170000E04F818
:10AB200038092146084600F06DF84FF00002EEB1FA
:10AB3000E06ED100C840A854A36ECB40A8180371A2
:10AB4000636ECB400372236ECB400373E36DCB4047
:10AB50000374A36DCB400375636DCB400376236D07
:10AB6000CB40521C0377042AE2D31FE01823504243
:10AB7000216D03EBC000C140A954666DC640A91801
:10AB80000E71A66DC6400E72E66DC6400E73266E3F
:10AB9000C6400E74666EC6400E75A66EC6400E7632
:10ABA000E66EC640521C0E77042AE0D3002070BD2A
:10ABB000A8B100210164C0E912110A4901650A49DE
:10ABC00041650A4981650A49C1650A4901660A4920
:10ABD00041660A4981660A49C166002070470E2015
:10ABE0007047000067E6096A85AE67BB72F36E3C8A
:10ABF0003AF54FA57F520E518C68059BABD9831F48
:10AC000019CDE05B2DE9F04FC8B0002213466F4626
:10AC1000CC181B1D2568E4782DBA25F0FF052543C7
:10AC200047F82250521C102AF2D31BE007EB820196
:10AC300051F8083C4FEA734484EAF34484EA9324CD
:10AC400051F83C3C4FEAF31585EAB34585EAD30356
:10AC5000234451F81C4C51F8401C2144194447F836
:10AC60002210521C402AE1D3036D4793416D469157
:10AC7000846D4594C26D44929246026E4392456E35
:10AC80004295A946856E4195C66E4096B34600260C
:10AC90004FEAB21787EAF22787EA726C02EA0907DD
:10ACA00025EA020887EA0807BC44204F57F82680A7
:10ACB00008EB0B07BC445DF82670AB460CEB070EA7
:10ACC0004FEAB30787EA733787EAB35C81EA040780
:10ACD0004D4601EA040891461F400AEB0E02A246C7
:10ACE00087EA08070C46BC441946761C0EEB0C0399
:10ACF000402ECDD3479E33440365469B194441659E
:10AD000045992144816544995144C1654399114451
:10AD100001664299494441664199294481664099B6
:10AD20005944C16648B0BDE8F08F000090BB0700F1
:10AD30002DE9F04116460F46040004D006B317B1C2
:10AD40000025A8461AE00E20BDE8F081216C785D50
:10AD50006054206C401C206440280ED121460846D7
:10AD6000FFF750FFD4E912014FF40072801841F14F
:10AD70000001C4F84080C4E912016D1CB542E5D35E
:10AD80000020E1E710B51620F7F7E6FF48B10C48C0
:10AD900082684FF4800152B1016821F480010160A2
:10ADA00010BDBDE8104042F20100F8F71DB94FF0A8
:10ADB000E020C0F88011BFF34F8FBFF36F8F10BD3D
:10ADC000B07D00202DE9F04100F500521A481B4FDC
:10ADD0000123C01B174CC008556803EB0040A54277
:10ADE00001D017491FE04D1EC5F30B05491B41F665
:10ADF000FF75966829448E4201D2124913E04FF440
:10AE000040514D68A54211D10C78102C01D9096927
:10AE100000E000211478102C01D9126900E0002212
:10AE2000914203D00849FDF7B5F900231846BDE863
:10AE3000F0810000DBE5B15168CE070038CE070095
:10AE400024C40700B8C3070004C3070010B51620C8
:10AE5000F7F782FFA0B1114890F8000440090828D4
:10AE600011D20121814011F0EC0F0CD00C48826806
:10AE70004FF480016AB1016841F48001016010BDA6
:10AE800042F2010001E042F20200BDE81040F8F792
:10AE9000ABB84FF0E020C0F8001110BD16E000E0A4
:10AEA000B07D00202DE9F0471E46924689460546B2
:10AEB000040C089FF9F7E4FB8046FDF70BFAA0426B
:10AEC00004D80FA140F2A910F8F760FA44EA08414B
:10AED000741C1B483C4000EB84023E4000EB8600A3
:10AEE000D160C16865F3C5016AF3891169F39F21D7
:10AEF00021F00301491C21F00401C160BDE8F08785
:10AF00002E2E5C2E2E5C2E2E5C2E2E5C2E2E5C6346
:10AF10006F6D706F6E656E74735C6C696272617276
:10AF20006965735C6C6F675C7372635C6E72665F9D
:10AF30006C6F675F66726F6E74656E642E6300007F
:10AF4000548100202DE9FC47814616481746884663
:10AF500005681C46012201A91846F9F7ABF8124E04
:10AF6000B8B101998B1C00200AE000BF57F82020DF
:10AF700003EA050C06EB8C0C401C5B1CCCF80C2087
:10AF8000A042F3D30B462246414648460095FFF7C0
:10AF900089FF307802E000BFFCF78CFF0028FBD16E
:10AFA000BDE8FC87145A0020548100202DE9FF41A0
:10AFB000324800F15C01826B6846FEF75DFF304F5E
:10AFC0009DE8070007F11C032F4C83E80700194692
:10AFD0002C48C8600020A0706060A0604FF44771EA
:10AFE000A7F54070F6F735FAA7F54072274902F544
:10AFF0004770FEF7B0FC2649264A891AC908012283
:10B0000002EB014578B1A07838B1A7F5407090F80F
:10B010006C110029017826D041B128461EA100BF3D
:10B02000FDF7B8F828E0284623A1F9E790F8720167
:10B0300010B3D4E901122C4E6846FEF71DFF9DE8BF
:10B040000F001C3787E80F004FF4B2713046F6F757
:10B0500000FA3246254906F5D470FEF77CFC30B97B
:10B06000284623A1DCE739B1807928B12F4E012091
:10B07000E66004B0BDE8F0810020FAE73C760020ED
:10B08000BC7C0020899C0700DC59002060B80700C8
:10B0900068CE070038CE070048616E646C65723A6E
:10B0A00020496E76616C696420696E697420636FF3
:10B0B0006D6D616E642E000048616E646C65723A5D
:10B0C00020496E76616C69642070726F746F636F73
:10B0D0006C20627566666572206D5F70625F737466
:10B0E0007265616D00000000307B002040B70700F2
:10B0F00048616E646C65723A20496E76616C696471
:10B100002070726F746F636F6C2062756666657213
:10B11000206D5F70625F73747265616D2028696E67
:10B12000697420636F6D6D616E642900C4790020BD
:10B130002DE9F0410F460546234824492A46401A86
:10B14000C008042101EB004021A1FDF727F8B7F169
:10B15000807F03D324498F20F8F718F9962F03D264
:10B1600021499020F8F712F96FF07F40874200D212
:10B1700038461E4ED6F804150144381A21F07F4493
:10B18000411E6860952902D29630963C68602D7BFE
:10B19000042D03D314497720F8F7F8F806EB85005F
:10B1A000C0F8404512494FF4F86088474FF4A0704A
:10B1B00000EB85013046FDF735FA4FF48030A840AA
:10B1C000C6F80403BDE8F08188CE070038CE07003A
:10B1D00074696D65725F6163746976617465202856
:10B1E000307825782900000054BE07000040024056
:10B1F000B1B6070070B5174E3078002829D116482F
:10B2000000680125C0F3004008B914480560144CDB
:10B210004FF480712046FDF705FA4FF4A0712046E7
:10B22000FDF700FA4FF4A2712046FDF7FBF90D4A35
:10B230000020A02182F800140A4A1021203AC2F806
:10B240000011C4F80805A56025600220C4F80403B5
:10B25000357070BD7059002018040040080000408F
:10B260000040024024E000E070B515460E4604465A
:10B27000FFF7C0FF314620462560BDE87040FFF76C
:10B2800057BF000010B5044609480A492246401A33
:10B29000C008042101EB004007A1FCF77FFF217BE0
:10B2A0004FF4803088400949C1F8080310BD000000
:10B2B00088CE070038CE070074696D65725F7374BD
:10B2C0006F70202830782578290000000040024067
:10B2D0000870020A4A70020C8A70000EC8700420BE
:10B2E0007047000010B50248F9F7C1FE002010BDFC
:10B2F000FC59002010B514210448F6F7AAF80448B8
:10B300000068F9F76DFE002010BD0000A87F002046
:10B3100024BA07002DE9F05F8346DDE90A4A994621
:10B3200090460D460846012703E000BFB0FBF8F049
:10B330007F1C4045FAD2B94500D94F465FEACA7032
:10B3400012D18CB15FEA8A7002D5B9F1000F01D039
:10B35000202607E0302605E031465846641EF8F7FF
:10B3600003FF0CB1A742F7D35FF00106B9F1010F5B
:10B3700002D9A9F1010903E0B5FBF6F0404502D37B
:10B3800006FB08F6F2E7DFF83C9000BFB5FBF6F0ED
:10B3900000FB165519F800105846F8F7E5FEB6FB05
:10B3A000F8F6002EF2D15FEACA7009D0002C07D05F
:10B3B000A74205D220215846641EF8F7D5FEF5E7CE
:10B3C000BDE8F09FE8B907002DE9F04108460124E7
:10B3D0001646254600212B460A46FAF719FD0C4968
:10B3E0000C4A891ACF0830B105EB07400AA1FCF7D7
:10B3F000D1FE042409E0FAF7F1FC02463060042093
:10B4000000EB07400BA1FCF7C9FE2046BDE8F08128
:10B4100068CE070038CE070043616E277420666946
:10B420006E6420726F6F6D20666F7220757064613C
:10B430007465000057726974652061646472657395
:10B44000732073657420746F20307825303878004D
:10B450002DE9F0411C4B1D4F0F2600240125DB1B5D
:10B4600090F85520DB0805EB03450AB1042A03D107
:10B4700090F86430012B06D0D30707D090F85630EF
:10B48000012B02D002E0846E0DE0846D92070AD594
:10B4900090F85C20012A06D1026E0D48C0F5FC230D
:10B4A0009A4204D814443CB101260C6008E02846B6
:10B4B00008A1FCF77AFE042628460EA1FCF76AFED6
:10B4C0003046BDE8F081000068CE070038CE0700A6
:10B4D00000100700424C2073697A652028256429F2
:10B4E000206F766572206C696D6974202825642947
:10B4F00000000000496E6974207061636B65742000
:10B50000646F6573206E6F7420636F6E7461696E13
:10B510002076616C6964206669726D77617265205E
:10B5200073697A650000000030B1006805498842FF
:10B5300005D048F20250704748F201507047002091
:10B54000704700006E52464870B5FDF78DFB00282D
:10B5500011D00020084A094B094C0121166801FA54
:10B5600000F52E4203D004EB8005C5F80036401CE0
:10B57000C0B20728F2D370BD080501403546526EAF
:10B58000000001400748084910B5401AC0080321CF
:10B5900001EB004005A1FCF7FDFDBDE81040FFF701
:10B5A000D3BF000038CE070038CE0700496E74655F
:10B5B000726E616C20666565640000000020704753
:10B5C000002070472DE9FC4180461C4617460E4678
:10B5D0000C48089DF9F754FD10B11120BDE8FC811D
:10B5E000A20839463046FCF7E7FF0648F9F73FFD69
:10B5F00033463A4601214046CDE90045F9F794F833
:10B600000020EBE7FC5900202DE9F84F114D88464A
:10B6100081461E4617466946DDF828A02868F9F7D6
:10B62000FAFC040013D01C21F5F713FF0020207151
:10B63000C4F80090C4E90486C4E902A769462868F2
:10B64000F9F70AFDFEF7CCFE0020BDE8F88F0420D4
:10B65000FBE7000024BA0700000000000000000023
:10B660000338FDD8704700007EF8C9F6120F4CD79A
:10B670009208C17183F5768FE216ECBA29939A7419
:10B6800003F32B069BFC932EF7111725792DB9D6C2
:10B69000BE74B76C6731C8341D64FD04B795B1DC66
:10B6A000017F21F1461AF08B00000000000000002D
:10B6B0000338FDD8704700005D8C0700638C0700DD
:10B6C000398C070020000000780000000000000016
:10B6D0004800280000204000B917070000000000C3
:10B6E0000100010000000000010000000000000057
:10B6F0000200050001000000220000000000000020
:10B700000000000000000000000000000000000039
:10B710000100010000000000010000000000000026
:10B7200002000500010000004200000000000000CF
:10B730000000000000000000000000000000000009
:10B74000010011000400FCFF0400000000000000E4
:10B75000020011000400FCFF0400000000000000D3
:10B76000030021000400FCFF0400100000000000A2
:10B77000040011000100FFFF0100000000000000B4
:10B78000050011000200FEFF0400000000000000A0
:10B79000060011000400FCFF04000000000000008F
:10B7A000070011000400FCFF04000000000000007E
:10B7B000080017000200FEFF24000000E0B60700AA
:10B7C000090010000100FFFF01000000DCB60700C7
:10B7D0000A0027000200FEFF4400030010B7070024
:10B7E0000000000000000000000000000000000059
:10B7F000010011000100FFFF010000000000000037
:10B80000020017000200FEFF6401000040B70700BD
:10B810000000000000000000000000000000000028
:10B82000010007000000000068010000F0B70700F9
:10B830000200010000000000010000000000000004
:10B8400003000500010000004200000000000000AD
:10B8500000000000000000000000000000000000E8
:10B86000010017000400FCFF68010000F0B70700AA
:10B87000020017000400FCFFAC01000020B8070024
:10B8800000000000000000000000000000000000B8
:10B89000001103000011130002000000010000006D
:10B8A0000338FDD870470C000C000000580200005F
:10B8B0000200000000000000020000000000000084
:10B8C000A45E00200900000000000000000000004D
:10B8D000010000000000000028000000000000003F
:10B8E0000000000000010000000001000000000056
:10B8F0000000000000000000000000000000000048
:10B90000E535070000000000000000000000000016
:10B910000200000000000100000000000000000024
:10B920000800000000000000E5350700E195070071
:10B930000000000000000000040000000000000003
:10B9400000000000000000000000000000000000F7
:10B9500000000000000000000000000000000000E7
:10B96000F4000000000000001800000000000000CB
:10B9700000000000000000000000000000000000C7
:10B9800000000000000000000000000000000000B7
:10B99000170000000000000050EADA308883B89FEA
:10B9A000604F15F30000C98E020000000000000087
:10B9B0000000000000000000040000000000000083
:10B9C0000000000000000000000000000000000077
:10B9D0000001000000000000000000000000000066
:10B9E00000000000000000003031323334353637BB
:10B9F000383941424344454600100000040000002D
:10BA000001000000F14A0700E5B2070005A40700A5
:10BA1000C5B5070095460700D9A40700BDB50700C6
:10BA2000114C0700BC7D0020001000000400000045
:10BA300001000000FD4A0700F5B2070013A407004B
:10BA400009B60700DD460700DDA40700C1B5070001
:10BA5000214C0700556E6B6E6F776E206572726FAA
:10BA60007220636F64650000000000001CC90700BD
:10BA700001000000C8C7070002000000BCC50700A5
:10BA8000030000003CC807000400000090C8070045
:10BA90000500000070C70700060000000CC7070083
:10BAA0000700000078C807000800000084C70700EE
:10BAB00009000000E8C707000A00000004C90700E9
:10BAC0000B000000A4C507000C0000009CC7070085
:10BAD0000D0000006CC907000E00000068C80700D8
:10BAE0000F000000A4C8070010000000D8C807001D
:10BAF0001100000080C907001200000054C90700AF
:10BB000013000000F0C807008000000024C70700F1
:10BB10008100000060C607008200000020C6070008
:10BB20008300000000C60700840000003CC6070038
:10BB30008500000048C707008600000050C80700C5
:10BB400090000000ECC6070091000000E0C507006F
:10BB500092000000B0C7070000820000B8C80700CC
:10BB60000182000004C807000282000020C807000C
:10BB7000008400007CC607000184000028C907007B
:10BB800002840000C4C6070003840000A0C60700AA
:10BB9000982F8A4291443771CFFBC0B5A5DBB5E938
:10BBA0005BC25639F111F159A4823F92D55E1CABAC
:10BBB00098AA07D8015B8312BE853124C37D0C553A
:10BBC000745DBE72FEB1DE80A706DC9B74F19BC182
:10BBD000C1699BE48647BEEFC69DC10FCCA10C2472
:10BBE0006F2CE92DAA84744ADCA9B05CDA88F97656
:10BBF00052513E986DC631A8C82703B0C77F59BFC0
:10BC0000F30BE0C64791A7D55163CA0667292914EB
:10BC1000850AB72738211B2EFC6D2C4D130D385388
:10BC200054730A65BB0A6A762EC9C281852C72924A
:10BC3000A1E8BFA24B661AA8708B4BC2A3516CC778
:10BC400019E892D1240699D685350EF470A06A10B1
:10BC500016C1A419086C371E4C774827B5BCB03400
:10BC6000B30C1C394AAAD84E4FCA9C5BF36F2E689E
:10BC7000EE828F746F63A5781478C8840802C78C2D
:10BC8000FAFFBE90EB6C50A4F7A3F9BEF27871C630
:10BC9000797D0700777D0700717D070000000000B7
:10BCA0000338FDD870470000BC8000207F000000F2
:10BCB0003C810020D8CE0700E0CE07000000000045
:10BCC0000000000000100201B4BC0700C4BC070063
:10BCD00008000000ECBC0700FCBC070008000000E6
:10BCE000FCBC07000CBD070008000000F8CE0700F0
:10BCF00000CF07000000000000000000E8CE0700B1
:10BD0000F8CE070000000000000000000000000066
:10BD1000000000000000000000000000D0CE07007E
:10BD2000D8CE070000000000000000006859002085
:10BD30000CBD07002CBD070008000000E0CE070086
:10BD4000E8CE070000000000000000003CBD070036
:10BD50004CBD070008000000FD980700A5980700EB
:10BD60004D980700C3970700C99707008197070000
:10BD7000CF9707000D9807000000000000404040EA
:10BD800040404040404041414141414040404040AE
:10BD9000404040404040404040404040400502025A
:10BDA0000202020202020202020202020220202019
:10BDB0002020202020202002020202020202909075
:10BDC0009090909010101010101010101010101073
:10BDD00010101010101010100202020202028888C7
:10BDE00088888888080808080808080808080808D3
:10BDF00008080808080808080202020240000000BB
:10BE00007DBD07002E2E5C2E2E5C2E2E5C2E2E5C11
:10BE10002E2E5C636F6D706F6E656E74735C6C69F3
:10BE2000627261726965735C626F6F746C6F61647A
:10BE300065725C6E72665F626F6F746C6F61646571
:10BE4000725F6170705F73746172745F66696E6156
:10BE50006C2E63002E2E5C2E2E5C2E2E5C2E2E5C05
:10BE60002E2E5C636F6D706F6E656E74735C6C69A3
:10BE7000627261726965735C626F6F746C6F61642A
:10BE800065725C6E72665F626F6F746C6F61646521
:10BE9000725F6466755F74696D6572732E6300000E
:10BEA0002E2E5C2E2E5C2E2E5C2E2E5C2E2E5C6397
:10BEB0006F6D706F6E656E74735C6C6962726172C7
:10BEC0006965735C626F6F746C6F616465725C6EE0
:10BED00072665F626F6F746C6F616465725F6677C4
:10BEE0005F61637469766174696F6E2E6300000030
:10BEF00043524320636F6D7075746174696F6E2077
:10BF00006661696C656420666F7220636F70696535
:10BF100064206170703A20737263206372633A2008
:10BF20003078253038782C20726573206372633A3C
:10BF300020307825303878004120536F667444658E
:10BF40007669636520686173206A75737420626521
:10BF5000656E206163746976617465642E2049742E
:10BF60002773206C696B656C79207468617420613B
:10BF70006E206170706C69636174696F6E2077699F
:10BF80006C6C20636F6D6520696D6D6564696174AB
:10BF9000656C7900526563656976656420424C453D
:10BFA0005F47415454535F4556545F455843484199
:10BFB0004E47455F4D54555F5245515545535420AA
:10BFC00028726571756573743A2025642C2072653A
:10BFD000706C793A202564292E0000002E2E5C2EEC
:10BFE0002E5C2E2E5C2E2E5C2E2E5C636F6D706F81
:10BFF0006E656E74735C6C69627261726965735CA4
:10C00000626F6F746C6F616465725C626C655F64B3
:10C0100066755C6E72665F6466755F626C652E63E2
:10C02000000000006E72665F6673746F7261676510
:10C030005F777269746528616464723D25702C2095
:10C040007372633D25702C206C656E3D2564206203
:10C0500079746573292C2071756575652075736118
:10C0600067653A20256400004372656174696E67F4
:10C0700020746865206F626A6563742077697468EC
:10C080002073697A652030782530387820776F758D
:10C090006C64206F766572666C6F77206669726D6E
:10C0A000776172652073697A652E204F66667365C5
:10C0B000742069732030782530387820616E6420D0
:10C0C0006669726D776172652073697A652069733C
:10C0D000203078253038782E000000002E2E5C2E7F
:10C0E0002E5C2E2E5C2E2E5C2E2E5C636F6D706F80
:10C0F0006E656E74735C6C69627261726965735CA3
:10C10000626F6F746C6F616465725C6466755C6E9F
:10C1100072665F6466755F7265715F68616E646C9C
:10C1200065722E6300000000526573657474696E59
:10C130006720626F6F746C6F6164657220736574E1
:10C1400074696E67732073696E6365206E656974C8
:10C15000686572207468652073657474696E6773AE
:10C160002070616765206E6F72207468652062615F
:10C17000636B7570206172652076616C696420283C
:10C18000435243206572726F72292E005265737498
:10C190006F72696E672073657474696E6773206669
:10C1A000726F6D206261636B75702073696E636579
:10C1B000207468652073657474696E67732070619C
:10C1C000676520636F6E74656E747320617265209D
:10C1D000696E76616C6964202843524320657272EF
:10C1E0006F72292E0000000044657374696E6174DB
:10C1F000696F6E2073657474696E67732061726510
:10C20000206964656E746963616C20746F20736F5C
:10C21000757263652C207772697465206E6F742067
:10C220006E65656465642E20536B697070696E6716
:10C230002E0000002E2E5C2E2E5C2E2E5C2E2E5CF0
:10C240002E2E5C636F6D706F6E656E74735C6C69BF
:10C25000627261726965735C626F6F746C6F616446
:10C2600065725C6466755C6E72665F6466755F734A
:10C27000657474696E67732E630000002E2E5C2E49
:10C280002E5C2E2E5C2E2E5C2E2E5C636F6D706FDE
:10C290006E656E74735C6C69627261726965735C01
:10C2A000626F6F746C6F616465725C6466755C6EFE
:10C2B00072665F6466755F7574696C732E630000E7
:10C2C0004D616A6F722053442075706461746520FB
:10C2D000627574206E6F20424C2E2041626F727422
:10C2E00020746F2061766F696420696E636170618C
:10C2F0006369746174696E672074686520424C2EAE
:10C3000000000000546865206E657720536F6674E6
:10C31000446576696365206973206F6620612064D7
:10C320006966666572656E742066616D696C7920F8
:10C330007468616E207468652070726573656E74D0
:10C3400020536F66744465766963652E20436F6D74
:10C350007061746962696C6974792063616E6E6F73
:10C36000742062652067756172616E746565642E04
:10C3700000000000426F6F742076616C6964617424
:10C38000696F6E206F6620626F6F746C6F61646599
:10C3900072206973206E6F7420737570706F727481
:10C3A000656420616E642077696C6C206265206929
:10C3B000676E6F7265642E0054686520536F6674F3
:10C3C0004465766963652073697A6520696E2074B7
:10C3D000686520696E666F20737472756374206976
:10C3E0007320746F6F20736D616C6C20636F6D7060
:10C3F0006172656420776974682074686520736968
:10C400007A65207265706F7274656420696E20743D
:10C41000686520696E697420636F6D6D616E642E4E
:10C420000000000054686520536F667444657669A7
:10C43000636520646F6573206E6F7420636F6E7424
:10C4400061696E20746865206D61676963206E752F
:10C450006D626572206964656E74696679696E677C
:10C46000206974206173206120536F66744465767F
:10C470006963652E00000000496E76616C69646135
:10C4800074696E67206170702062656361757365A1
:10C4900020697420697320696E636F6D70617469BF
:10C4A000626C6520776974682074686520536F66D4
:10C4B000744465766963652E000000002E2E5C2EA4
:10C4C0002E5C2E2E5C2E2E5C2E2E5C636F6D706F9C
:10C4D0006E656E74735C6C69627261726965735CBF
:10C4E000626F6F746C6F616465725C6466755C6EBC
:10C4F00072665F6466755F76616C69646174696FAA
:10C500006E2E63002E2E5C2E2E5C2E2E5C2E2E5C4C
:10C510002E2E5C636F6D706F6E656E74735C6C69EC
:10C52000627261726965735C626F6F746C6F616473
:10C5300065725C6466755C6E72665F6466755F7674
:10C5400065725F76616C69646174696F6E2E6300F9
:10C550002E2E5C2E2E5C2E2E5C2E2E5C2E2E5C63E0
:10C560006F6D706F6E656E74735C6C696272617210
:10C570006965735C6578706572696D656E74616C10
:10C580005F73656374696F6E5F766172735C6E7200
:10C59000665F73656374696F6E5F697465722E633D
:10C5A000000000004E52465F4552524F525F494EC6
:10C5B00056414C49445F4441544100004E52465F4D
:10C5C0004552524F525F534F465444455649434596
:10C5D0005F4E4F545F454E41424C454400000000C1
:10C5E0004E52465F4552524F525F46454154555256
:10C5F000455F4E4F545F454E41424C45440000005C
:10C600004E52465F4552524F525F4D555445585F0A
:10C61000554E4C4F434B5F4641494C45440000004A
:10C620004E52465F4552524F525F4D555445585FEA
:10C630004C4F434B5F4641494C4544004E52465F88
:10C640004552524F525F4D555445585F434F4E44EB
:10C650005F494E49545F4641494C45440000000043
:10C660004E52465F4552524F525F4D555445585FAA
:10C67000494E49545F4641494C4544004E52465F3D
:10C680004552524F525F424C455F495053505F52A2
:10C69000585F504B545F5452554E434154454400EB
:10C6A0004E52465F4552524F525F424C455F495091
:10C6B00053505F504545525F52454A4543544544A7
:10C6C000000000004E52465F4552524F525F424CAE
:10C6D000455F495053505F4C494E4B5F444953436B
:10C6E0004F4E4E4543544544000000004E52465FB5
:10C6F0004552524F525F4150495F4E4F545F494D32
:10C70000504C454D454E5445440000004E52465F46
:10C710004552524F525F4E4F545F535550504F52F7
:10C72000544544004E52465F4552524F525F4D4F62
:10C7300044554C455F4E4F545F494E495449414C16
:10C74000495A4544000000004E52465F4552524F40
:10C75000525F4D4F44554C455F414C524541445901
:10C760005F494E495449414C495A45440000000034
:10C770004E52465F4552524F525F4E4F545F464FA6
:10C78000554E44004E52465F4552524F525F494EFD
:10C7900056414C49445F5354415445004E52465F04
:10C7A0004552524F525F444154415F53495A4500EC
:10C7B0004E52465F4552524F525F494F5F50454E71
:10C7C00044494E47000000004E52465F4552524FCA
:10C7D000525F5356435F48414E444C45525F4D496A
:10C7E0005353494E470000004E52465F4552524F48
:10C7F000525F494E56414C49445F4C454E47544860
:10C80000000000004E52465F4552524F525F445264
:10C81000565F5457495F4552525F414E41434B006A
:10C820004E52465F4552524F525F4452565F5457E4
:10C83000495F4552525F444E41434B004E52465F62
:10C840004552524F525F494E5445524E414C0000A2
:10C850004E52465F4552524F525F53544F524147DA
:10C86000455F46554C4C00004E52465F4552524F74
:10C87000525F4E554C4C00004E52465F4552524F4F
:10C88000525F494E56414C49445F504152414D0020
:10C890004E52465F4552524F525F4E4F5F4D454D8F
:10C8A000000000004E52465F4552524F525F464FC5
:10C8B0005242494444454E004E52465F4552524F03
:10C8C000525F4452565F5457495F4552525F4F562C
:10C8D000455252554E0000004E52465F4552524F4F
:10C8E000525F494E56414C49445F41444452000016
:10C8F0004E52465F4552524F525F5245534F55522A
:10C90000434553004E52465F4552524F525F494E87
:10C9100056414C49445F464C414753004E52465F96
:10C9200053554343455353004E52465F4552524F71
:10C93000525F424C455F495053505F4348414E4E11
:10C94000454C5F414C52454144595F455849535409
:10C95000530000004E52465F4552524F525F434FC4
:10C960004E4E5F434F554E54000000004E52465FFE
:10C970004552524F525F54494D454F5554000000A7
:10C980004E52465F4552524F525F42555359000036
:10C990002E2E5C2E2E5C2E2E5C2E2E5C2E2E5C639C
:10C9A0006F6D706F6E656E74735C6C6962726172CC
:10C9B0006965735C6C6F675C7372635C6E72665FF3
:10C9C0006C6F675F64656661756C745F6261636BF1
:10C9D000656E64732E6300007761726E696E670026
:10C9E00064656275670000001B5B313B33306D008E
:10C9F0001B5B306D000000001B5B313B33316D0071
:10CA00001B5B313B33326D001B5B313B33336D00BD
:10CA10001B5B313B33346D001B5B313B33356D00A9
:10CA20001B5B313B33366D001B5B313B33376D0095
:10CA3000696E666F000000006572726F7200000020
:10CA40002E2E5C2E2E5C2E2E5C2E2E5C2E2E5C63EB
:10CA50006F6D706F6E656E74735C6C69627261721B
:10CA60006965735C6578706572696D656E74616C1B
:10CA70005F73656374696F6E5F766172735C6E720B
:10CA8000665F73656374696F6E5F697465722E6843
:10CA90000000000073645F626C655F6366675F73CC
:10CAA000657428292072657475726E65642025731B
:10CAB000207768656E20617474656D7074696E6747
:10CAC00020746F2073657420424C455F4741545475
:10CAD000535F4346475F534552564943455F43487A
:10CAE000414E4745442E000073645F626C655F638E
:10CAF00066675F73657428292072657475726E6548
:10CB000064202573207768656E20617474656D708C
:10CB100074696E6720746F2073657420424C455FA2
:10CB2000434F4D4D4F4E5F4346475F56535F5555FC
:10CB300049442E0073645F626C655F6366675F7370
:10CB4000657428292072657475726E65642025737A
:10CB5000207768656E20617474656D7074696E67A6
:10CB600020746F2073657420424C455F47415454D4
:10CB7000535F4346475F415454525F5441425F53B1
:10CB8000495A452E0000000073645F626C655F6364
:10CB900066675F73657428292072657475726E65A7
:10CBA00064202573207768656E20617474656D70EC
:10CBB00074696E6720746F2073657420424C455F02
:10CBC000434F4E4E5F4346475F4741502E000000A3
:10CBD00073645F626C655F6366675F736574282961
:10CBE0002072657475726E656420257320776865A0
:10CBF0006E20617474656D7074696E6720746F2047
:10CC000073657420424C455F4741505F4346475F20
:10CC1000524F4C455F434F554E542E0073645F6234
:10CC20006C655F6366675F7365742829207265743D
:10CC300075726E6564202573207768656E20617457
:10CC400074656D7074696E6720746F2073657420ED
:10CC5000424C455F434F4E4E5F4346475F4741540A
:10CC6000542E00006E72665F626F6F746C6F616449
:10CC700065725F77647400006E72665F6466755FEC
:10CC8000626C65006E72665F6466755F666C617388
:10CC9000680000006E72665F6466755F7265715F42
:10CCA00068616E646C6572006E72665F6466755F63
:10CCB00073657474696E6773000000006E72665F5E
:10CCC0006466755F73657474696E67735F737663AA
:10CCD000690000006E72665F6466755F76616C69FC
:10CCE000646174696F6E00006E72665F6466755F82
:10CCF0007665725F76616C69646174696F6E00005D
:10CD00006D656D5F6D6E6772000000006E72665F2C
:10CD10006673746F72616765000000007274745FFF
:10CD20006C6F675F6261636B656E64006170700059
:10CD30006E72665F736468006E72665F7364685FCC
:10CD4000626C65006E72665F7364685F736F630028
:10CD500008200001FFFFFFFFFFFFFFFFFFFFFFFFB6
:10CD600000000000000000000000000001000000C2
:10CD7000FFFFFFFF512563FCC2CAB9F3849E17A7CA
:10CD8000ADFAE6BCFFFFFFFFFFFFFFFF0000000062
:10CD9000FFFFFFFF96C298D84539A1F4A033EB2DD1
:10CDA000817D0377F240A463E5E6BCF847422CE1BD
:10CDB000F2D1176BF551BF376840B6CBCE5E316B01
:10CDC0005733CE2B169E0F7C4AEBE78E9B7F1AFEC5
:10CDD000E242E34F4B60D2273E3CCE3BF6B053CC11
:10CDE000B0061D65BC86987655BDEBB3E7933AAAAD
:10CDF000D835C65A65160700FF2607001525070017
:10CE00000CCF0700685900201C0100003A2D0700D4
:10CE100028D00700845A00207C5700004A2D0700C4
:10CE2000E13707000537070090BC0700000000004D
:10CE30001CCD07000C5A002064CC0700000004043D
:10CE400078CC07000000040484CC07000000040430
:10CE500094CC070000000404A8CC070000000404E0
:10CE6000BCCC070000000404D4CC0700000004047C
:10CE7000E8CC07000000040400CD0700000000001B
:10CE80000CCD0700000004042CCD070000000404B2
:10CE900030CD07000000030338CD07000000030376
:10CEA00044CD070000000303B8590020F45E0020C1
:10CEB000055F0020085F0020F4000000205A0020D9
:10CEC000185A0020205A0020FC7F00201800000083
:10CED000D538070000000000F57A070000000000C8
:10CEE0002D7B070000000000A5880700000000005F
:10CEF000318A0700000000000D7B070000000000E1
:10CF000000000000030000004D6807000000000062
:10CF1000000000000000000080590020905900200F
:10CF20000000000000000000000000000000000001
:10CF300000000000000000000000000000000000F1
:10CF4000010000000000000000000000FF00FFFFE3
:10CF500000000000000000000000000000000000D1
:10CF600000000000000000000000000001000000C0
:10CF700000000000000000000000000000E00700CA
:10CF800000000000000000000000000000000000A1
:10CF90000000000000000000000000000000000091
:10CFA0000000000000000000000000000000000081
:10CFB00000000000FF000000FF0300000000000070
:10CFC0000000000000000000000000000000000061
:10CFD000000000000000000038CA0700D8C90700A0
:10CFE00030CA0700E0C90700F0C90700E8C9070018
:10CFF000F8C9070000CA070008CA070010CA0700DE
:10D0000018CA070020CA070028CA0700000000004D
:10D010000090D0030000000000000000F54407006D
:08D020000010000000000800F0
:020000041000EA
:0410140000100700C1
:020000041000EA
:0410180000E00700ED
:0400000500071201DD
:00000001FF
